******************************************************************************
             TMS320C2000 Linker PC v18.12.3                    
******************************************************************************
>> Linked Mon Jun 15 12:06:06 2020

OUTPUT FILE NAME:   <fcl_f2837x_tmdxiddk.out>
ENTRY POINT SYMBOL: "code_start"  address: 00000000


MEMORY CONFIGURATION

         name            origin    length      used     unused   attr    fill
----------------------  --------  ---------  --------  --------  ----  --------
  BEGIN                 00000000   00000002  00000002  00000000  RWIX
  BOOT_RSVD             00000002   000001ae  00000000  000001ae  RWIX
  RAMM0                 000001b0   00000250  00000000  00000250  RWIX
  RAMM1                 00000400   00000400  00000380  00000080  RWIX
  ADCA_RESULT           00000b00   00000020  00000000  00000020  RWIX
  ADCB_RESULT           00000b20   00000020  00000000  00000020  RWIX
  ADCC_RESULT           00000b40   00000020  00000000  00000020  RWIX
  ADCD_RESULT           00000b60   00000020  00000000  00000020  RWIX
  CPU_TIMER0            00000c00   00000008  00000000  00000008  RWIX
  CPU_TIMER1            00000c08   00000008  00000000  00000008  RWIX
  CPU_TIMER2            00000c10   00000008  00000000  00000008  RWIX
  PIE_CTRL              00000ce0   00000020  0000001a  00000006  RWIX
  PIE_VECT              00000d00   00000200  00000000  00000200  RWIX
  DMA                   00001000   00000200  00000000  00000200  RWIX
  CLA1                  00001400   00000040  00000000  00000040  RWIX
  CLA1_MSGRAMLOW        00001480   00000080  00000000  00000080  RWIX
  CLA1_MSGRAMHIGH       00001500   00000080  00000000  00000080  RWIX
  EPWM1                 00004000   00000100  00000000  00000100  RWIX
  EPWM2                 00004100   00000100  00000000  00000100  RWIX
  EPWM3                 00004200   00000100  00000000  00000100  RWIX
  EPWM4                 00004300   00000100  00000000  00000100  RWIX
  EPWM5                 00004400   00000100  00000000  00000100  RWIX
  EPWM6                 00004500   00000100  00000000  00000100  RWIX
  EPWM7                 00004600   00000100  00000000  00000100  RWIX
  EPWM8                 00004700   00000100  00000000  00000100  RWIX
  EPWM9                 00004800   00000100  00000000  00000100  RWIX
  EPWM10                00004900   00000100  00000000  00000100  RWIX
  EPWM11                00004a00   00000100  00000000  00000100  RWIX
  EPWM12                00004b00   00000100  00000000  00000100  RWIX
  ECAP1                 00005000   00000020  00000000  00000020  RWIX
  ECAP2                 00005020   00000020  00000000  00000020  RWIX
  ECAP3                 00005040   00000020  00000000  00000020  RWIX
  ECAP4                 00005060   00000020  00000000  00000020  RWIX
  ECAP5                 00005080   00000020  00000000  00000020  RWIX
  ECAP6                 000050a0   00000020  00000000  00000020  RWIX
  EQEP1                 00005100   00000040  00000000  00000040  RWIX
  EQEP2                 00005140   00000040  00000000  00000040  RWIX
  EQEP3                 00005180   00000040  00000000  00000040  RWIX
  DACA                  00005c00   00000010  00000000  00000010  RWIX
  DACB                  00005c10   00000010  00000000  00000010  RWIX
  DACC                  00005c20   00000010  00000000  00000010  RWIX
  CMPSS1                00005c80   00000020  00000000  00000020  RWIX
  CMPSS2                00005ca0   00000020  00000000  00000020  RWIX
  CMPSS3                00005cc0   00000020  00000000  00000020  RWIX
  CMPSS4                00005ce0   00000020  00000000  00000020  RWIX
  CMPSS5                00005d00   00000020  00000000  00000020  RWIX
  CMPSS6                00005d20   00000020  00000000  00000020  RWIX
  CMPSS7                00005d40   00000020  00000000  00000020  RWIX
  CMPSS8                00005d60   00000020  00000000  00000020  RWIX
  SDFM1                 00005e00   00000080  00000000  00000080  RWIX
  SDFM2                 00005e80   00000080  00000000  00000080  RWIX
  MCBSPA                00006000   00000040  00000000  00000040  RWIX
  MCBSPB                00006040   00000040  00000000  00000040  RWIX
  SPIA                  00006100   00000010  00000000  00000010  RWIX
  SPIB                  00006110   00000010  00000000  00000010  RWIX
  SPIC                  00006120   00000010  00000000  00000010  RWIX
  SPID                  00006130   00000010  00000000  00000010  RWIX
  UPP                   00006200   00000100  00000000  00000100  RWIX
  WD                    00007000   00000040  00000000  00000040  RWIX
  NMIINTRUPT            00007060   00000010  00000000  00000010  RWIX
  XINT                  00007070   00000010  00000000  00000010  RWIX
  SCIA                  00007200   00000010  00000000  00000010  RWIX
  SCIB                  00007210   00000010  00000000  00000010  RWIX
  SCIC                  00007220   00000010  00000000  00000010  RWIX
  SCID                  00007230   00000010  00000000  00000010  RWIX
  I2CA                  00007300   00000040  00000000  00000040  RWIX
  I2CB                  00007340   00000040  00000000  00000040  RWIX
  ADCA                  00007400   00000080  00000000  00000080  RWIX
  ADCB                  00007480   00000080  00000000  00000080  RWIX
  ADCC                  00007500   00000080  00000000  00000080  RWIX
  ADCD                  00007580   00000080  00000000  00000080  RWIX
  INPUT_XBAR            00007900   00000020  00000000  00000020  RWIX
  XBAR                  00007920   00000020  00000000  00000020  RWIX
  SYNC_SOC              00007940   00000010  00000000  00000010  RWIX
  DMACLASRCSEL          00007980   00000040  00000000  00000040  RWIX
  EPWM_XBAR             00007a00   00000040  00000000  00000040  RWIX
  CLB_XBAR              00007a40   00000040  00000000  00000040  RWIX
  OUTPUT_XBAR           00007a80   00000040  00000000  00000040  RWIX
  GPIOCTRL              00007c00   00000180  00000000  00000180  RWIX
  GPIODAT               00007f00   00000030  00000000  00000030  RWIX
  RAMLS0                00008000   00000800  00000000  00000800  RWIX
  RAMLS1                00008800   00000800  00000150  000006b0  RWIX
  RAMLS2                00009000   00000800  00000110  000006f0  RWIX
  RAMLS3                00009800   00000800  0000003a  000007c6  RWIX
  RAMLS4                0000a000   00000800  00000200  00000600  RWIX
  RAMLS5                0000a800   00000800  00000000  00000800  RWIX
  RAMLS6                0000b000   00000800  00000000  00000800  RWIX
  RAMLS7                0000b800   00000800  00000000  00000800  RWIX
  RAMD0                 0000c000   00000800  00000000  00000800  RWIX
  RAMD1                 0000c800   00000800  00000000  00000800  RWIX
  RAMGS0                0000d000   00001000  00001000  00000000  RWIX
  RAMGS1                0000e000   00001000  00001000  00000000  RWIX
  RAMGS2                0000f000   00001000  00001000  00000000  RWIX
  RAMGS3                00010000   00001000  00001000  00000000  RWIX
  RAMGS4                00011000   00001000  00001000  00000000  RWIX
  RAMGS5                00012000   00001000  00001000  00000000  RWIX
  RAMGS6                00013000   00001000  00001000  00000000  RWIX
  RAMGS7                00014000   00001000  00001000  00000000  RWIX
  RAMGS8                00015000   00001000  000006ca  00000936  RWIX
  RAMGS9                00016000   00001000  00000000  00001000  RWIX
  RAMGS10               00017000   00001000  00000000  00001000  RWIX
  RAMGS11               00018000   00001000  00000000  00001000  RWIX
  RAMGS12               00019000   00001000  00000f20  000000e0  RWIX
  RAMGS13               0001a000   00001000  00000d9d  00000263  RWIX
  RAMGS14               0001b000   00001000  0000098e  00000672  RWIX
  RAMGS15               0001c000   00001000  00000000  00001000  RWIX
  CPU1TOCPU2RAM         0003a000   00000800  00000000  00000800  RWIX
  CPU2TOCPU1RAM         0003b000   00000800  00000000  00000800  RWIX
  EMIF1                 00047000   00000800  00000000  00000800  RWIX
  EMIF2                 00047800   00000800  00000000  00000800  RWIX
  CANA                  00048000   00000800  00000000  00000800  RWIX
  CANA_MSG_RAM          00049000   00000800  00000000  00000800  RWIX
  CANB                  0004a000   00000800  00000000  00000800  RWIX
  CANB_MSG_RAM          0004b000   00000800  00000000  00000800  RWIX
  IPC                   00050000   00000024  00000000  00000024  RWIX
  FLASHPUMPSEMAPHORE    00050024   00000002  00000000  00000002  RWIX
  DEV_CFG               0005d000   00000180  00000000  00000180  RWIX
  ANALOG_SUBSYS         0005d180   00000080  00000000  00000080  RWIX
  CLK_CFG               0005d200   00000100  00000000  00000100  RWIX
  CPU_SYS               0005d300   00000100  00000000  00000100  RWIX
  ROMPREFETCH           0005e608   00000002  00000000  00000002  RWIX
  DCSM_Z1               0005f000   00000030  00000000  00000030  RWIX
  DCSM_Z2               0005f040   00000030  00000000  00000030  RWIX
  DCSM_COMMON           0005f070   00000010  00000000  00000010  RWIX
  MEMCFG                0005f400   00000080  00000000  00000080  RWIX
  EMIF1CONFIG           0005f480   00000020  00000000  00000020  RWIX
  EMIF2CONFIG           0005f4a0   00000020  00000000  00000020  RWIX
  ACCESSPROTECTION      0005f4c0   00000040  00000000  00000040  RWIX
  MEMORYERROR           0005f500   00000040  00000000  00000040  RWIX
  ROMWAITSTATE          0005f540   00000002  00000000  00000002  RWIX
  FLASH0_CTRL           0005f800   00000300  00000000  00000300  RWIX
  FLASH0_ECC            0005fb00   00000040  00000000  00000040  RWIX
  RESET                 003fffc0   00000002  00000000  00000002  RWIX


SECTION ALLOCATION MAP

 output                                  attributes/
section   page    origin      length       input sections
--------  ----  ----------  ----------   ----------------
codestart 
*          0    00000000    00000002     
                  00000000    00000002     F2837xD_CodeStartBranch.obj (codestart)

.cinit     0    00008800    00000150     
                  00008800    00000124     (.cinit..data.load) [load image, compression = lzss]
                  00008924    00000006     (__TI_handler_table)
                  0000892a    00000004     (.cinit..bss.load) [load image, compression = zero_init]
                  0000892e    00000004     (.cinit..bss_cla.load) [load image, compression = zero_init]
                  00008932    00000004     (.cinit.ClaData.load) [load image, compression = zero_init]
                  00008936    00000004     (.cinit.SFRA_F32_Data.load) [load image, compression = zero_init]
                  0000893a    00000002     --HOLE-- [fill = 0]
                  0000893c    00000014     (__TI_cinit_table)

.reset     0    003fffc0    00000000     DSECT

.stack     0    00000400    00000380     UNINITIALIZED
                  00000400    00000380     --HOLE--

.init_array 
*          0    0000d000    00000000     UNINITIALIZED

.bss       0    00019000    00000f20     UNINITIALIZED
                  00019000    0000044a     usb_ex7_host_msc.obj (.bss)
                  0001944a    00000100     usb_ex4_dev_bulk_structs.obj (.bss:g_pui8USBRxBuffer)
                  0001954a    00000100     usb_ex4_dev_bulk_structs.obj (.bss:g_pui8USBTxBuffer)
                  0001964a    00000100     fcl_tformat_f2837x_config.obj (.bss:tformatCRCtable)
                  0001974a    00000032     usblib_eabi.lib : usbdenum.obj (.bss:g_psDCDInst)
                  0001977c    00000004     ff.obj (.bss:FatFs$20)
                  00019780    0000009e     fcl_cpu_code.obj (.bss)
                  0001981e    0000008c     usblib_eabi.lib : usbdma.obj (.bss:g_psUSBDMAInst)
                  000198aa    00000080     usb_ex7_host_msc.obj (.bss:g_pHCDPool)
                  0001992a    00000064     fcl_f2837x_sfra_gui.obj (.bss:clMagVect)
                  0001998e    00000064     fcl_f2837x_sfra_gui.obj (.bss:clPhaseVect)
                  000199f2    00000064     fcl_f2837x_sfra_gui.obj (.bss:freqVect)
                  00019a56    00000064     fcl_f2837x_sfra_gui.obj (.bss:olMagVect)
                  00019aba    00000064     fcl_f2837x_sfra_gui.obj (.bss:olPhaseVect)
                  00019b1e    00000064     fcl_f2837x_sfra_gui.obj (.bss:plantMagVect)
                  00019b82    00000064     fcl_f2837x_sfra_gui.obj (.bss:plantPhaseVect)
                  00019be6    00000012     cmdline.obj (.bss:g_ppcArgv$13)
                  00019bf8    00000006     sfra_gui_scicomms_driverlib.obj (.bss:SFRA_GUI_cmdPacket)
                  00019bfe    00000002     usblib_eabi.lib : usbdenum.obj (.bss:g_ppsDevInfo)
                  00019c00    0000005a     fcl_f2837x_tmdxiddk.obj (.bss)
                  00019c5a    00000022     sfra_gui_scicomms_driverlib.obj (.bss)
                  00019c7c    00000004     usblib_eabi.lib : usbhostenum.obj (.bss:g_pui32Alloc)
                  00019c80    00000056     fcl_tformat_f2837x_config.obj (.bss)
                  00019cd6    00000050     usb_ex7_host_msc.obj (.bss:g_cTmpBuf$25)
                  00019d26    00000040     usb_ex7_host_msc.obj (.bss:g_cCmdBuf$25)
                  00019d66    00000040     usblib_eabi.lib : usbdenum.obj (.bss:g_pui8DataBufferIn)
                  00019da6    0000000c                     : usbtick.obj (.bss:g_pfnTickHandlers)
                  00019db2    0000000c                     : usbhostenum.obj (.bss:g_pi32USBHActiveDriver)
                  00019dbe    00000001     ff.obj (.bss)
                  00019dbf    00000001     --HOLE--
                  00019dc0    0000003e     usblib_eabi.lib : usbhhub.obj (.bss)
                  00019dfe    00000020     sfra_gui_scicomms_driverlib.obj (.bss:SFRA_GUI_arrayGetList)
                  00019e1e    00000020     sfra_gui_scicomms_driverlib.obj (.bss:SFRA_GUI_cmdDispatcher)
                  00019e3e    00000020     sfra_gui_scicomms_driverlib.obj (.bss:SFRA_GUI_dataSetList)
                  00019e5e    00000020     sfra_gui_scicomms_driverlib.obj (.bss:SFRA_GUI_varGetList)
                  00019e7e    00000020     sfra_gui_scicomms_driverlib.obj (.bss:SFRA_GUI_varSetBtnList)
                  00019e9e    00000020     sfra_gui_scicomms_driverlib.obj (.bss:SFRA_GUI_varSetSldrList)
                  00019ebe    00000020     sfra_gui_scicomms_driverlib.obj (.bss:SFRA_GUI_varSetTxtList)
                  00019ede    00000020     fcl_f2837x_sfra_gui.obj (.bss)
                  00019efe    0000000c     usblib_eabi.lib : usbhostenum.obj (.bss:g_ppvDriverInstance)
                  00019f0a    0000000c                     : usbtick.obj (.bss:g_pvTickInstance)
                  00019f16    00000006                     : usbmode.obj (.bss)
                  00019f1c    00000004     usb_ex4_dev_bulk.obj (.bss)

.init_array 
*          0    000001b0    00000000     UNINITIALIZED

.data      0    0001a000    00000d9d     UNINITIALIZED
                  0001a000    00000362     usblib_eabi.lib : usbhostenum.obj (.data)
                  0001a362    00000190     fcl_f2837x_tmdxiddk.obj (.data:DBUFF_4CH1)
                  0001a4f2    00000190     fcl_f2837x_tmdxiddk.obj (.data:DBUFF_4CH2)
                  0001a682    00000190     fcl_f2837x_tmdxiddk.obj (.data:DBUFF_4CH3)
                  0001a812    00000190     fcl_f2837x_tmdxiddk.obj (.data:DBUFF_4CH4)
                  0001a9a2    00000012     usblib_eabi.lib : usbdbulk.obj (.data:g_pui8BulkDeviceDescriptor)
                  0001a9b4    00000009                     : usbdbulk.obj (.data:g_pui8BulkDescriptor)
                  0001a9bd    00000001     fat_usbmsc.obj (.data)
                  0001a9be    00000002     rts2800_fpu32_eabi.lib : _lock.c.obj (.data:_lock)
                  0001a9c0    00000128     fcl_f2837x_tmdxiddk.obj (.data)
                  0001aae8    0000000e     fcl_f2837x_tmdxiddk.obj (.data:posEncElecTheta)
                  0001aaf6    00000008     fcl_f2837x_tmdxiddk.obj (.data:adcHandle)
                  0001aafe    00000002     scistdio.obj (.data)
                  0001ab00    00000106     fcl_cpu_code.obj (.data)
                  0001ac06    00000038     usb_ex7_host_msc.obj (.data:g_sFresultStrings)
                  0001ac3e    00000002     usb_ex7_host_msc.obj (.data)
                  0001ac40    00000064     usb_ex4_dev_bulk_structs.obj (.data)
                  0001aca4    00000050     usb_ex7_host_msc.obj (.data:g_cCwdBuf$25)
                  0001acf4    00000036     usb_ex7_host_msc.obj (.data:g_psCmdTable)
                  0001ad2a    00000020     PM_tformat_lib_f2837x.lib : pm_tformat_source.obj (.data:tformat_tile1HLCInstr)
                  0001ad4a    0000000e     fcl_f2837x_tmdxiddk.obj (.data:posEncMechTheta)
                  0001ad58    0000000e     usblib_eabi.lib : usbhmsc.obj (.data)
                  0001ad66    00000008     usb_ex4_dev_bulk.obj (.data)
                  0001ad6e    00000006     device.obj (.data)
                  0001ad74    00000006     fcl_f2837x_tmdxiddk.obj (.data:pwmHandle)
                  0001ad7a    00000006     rts2800_fpu32_eabi.lib : exit.c.obj (.data)
                  0001ad80    00000006     usblib_eabi.lib : usbtick.obj (.data)
                  0001ad86    00000004                     : usbdbulk.obj (.data:g_psBulkSections)
                  0001ad8a    00000004                     : usbmode.obj (.data)
                  0001ad8e    00000004     fcl_f2837x_tmdxiddk.obj (.data:vTimer0)
                  0001ad92    00000004     fcl_f2837x_tmdxiddk.obj (.data:vTimer1)
                  0001ad96    00000004     fcl_f2837x_tmdxiddk.obj (.data:vTimer2)
                  0001ad9a    00000002     usblib_eabi.lib : usbdenum.obj (.data)
                  0001ad9c    00000001     rts2800_fpu32_eabi.lib : errno.c.obj (.data)

.const     0    0001b000    0000098e     
                  0001b000    0000041a     <whole-program> (.const:.string)
                  0001b41a    0000007e     usblib_eabi.lib : usbdconfig.obj (.const:.string)
                  0001b498    0000007d                     : usbhostenum.obj (.const:.string)
                  0001b515    00000001     --HOLE-- [fill = 0]
                  0001b516    0000007c                     : usbdbulk.obj (.const:.string)
                  0001b592    0000007c                     : usbdenum.obj (.const:.string)
                  0001b60e    00000077                     : usbringbuf.obj (.const:.string)
                  0001b685    00000001     --HOLE-- [fill = 0]
                  0001b686    00000076                     : usbbuffer.obj (.const:.string)
                  0001b6fc    00000074                     : usbmode.obj (.const:.string)
                  0001b770    00000073                     : usbdma.obj (.const:.string)
                  0001b7e3    00000001     --HOLE-- [fill = 0]
                  0001b7e4    00000060     driverlib_eabi.lib : usb.obj (.const:.string)
                  0001b844    00000030     usb_ex4_dev_bulk_structs.obj (.const:g_pui8ConfigString)
                  0001b874    00000028     usb_ex4_dev_bulk_structs.obj (.const:g_pui8DataInterfaceString)
                  0001b89c    00000028     usb_ex4_dev_bulk_structs.obj (.const:g_pui8ProductString)
                  0001b8c4    00000024     usb_ex4_dev_bulk_structs.obj (.const:g_pui8ManufacturerString)
                  0001b8e8    00000017     usblib_eabi.lib : usbdbulk.obj (.const:g_pui8BulkInterface)
                  0001b8ff    00000001     --HOLE-- [fill = 0]
                  0001b900    00000024                     : usbdbulk.obj (.const)
                  0001b924    0000001a                     : usbdenum.obj (.const:g_psUSBDStdRequests)
                  0001b93e    00000012     usb_ex4_dev_bulk_structs.obj (.const:g_pui8SerialNumberString)
                  0001b950    0000000c     fcl_f2837x_tmdxiddk.obj (.const)
                  0001b95c    0000000c     usb_ex4_dev_bulk_structs.obj (.const:g_ppui8StringDescriptors)
                  0001b968    0000000c     <whole-program> (.const)
                  0001b974    00000008     usb_ex7_host_msc.obj (.const)
                  0001b97c    00000004     usb_ex7_host_msc.obj (.const:g_ppHostClassDrivers$25)
                  0001b980    00000008     usblib_eabi.lib : usbhmsc.obj (.const)
                  0001b988    00000004     usb_ex4_dev_bulk_structs.obj (.const:g_pui8LangDescriptor)
                  0001b98c    00000002     usblib_eabi.lib : usbdbulk.obj (.const:g_ppBulkConfigDescriptors)

ClaData    0    00009800    0000003a     UNINITIALIZED
                  00009800    0000003a     fcl_cpu_code.obj (ClaData)

CLAscratch 
*          0    00009000    00000100     UNINITIALIZED
                  00009000    00000100     --HOLE--

SFRA_F32_Data 
*          0    00012000    00000022     UNINITIALIZED
                  00012000    00000022     sfra_f32_tmu_eabi.lib : sfra_f32_tmu_config_reset.obj (SFRA_F32_Data)

.bss_cla   0    00009100    00000010     UNINITIALIZED
                  00009100    0000000e     fcl_cla_code.obj (.bss_cla:Q_cla)
                  0000910e    00000002     fcl_cla_code.obj (.bss_cla:ClaQep)

Cla1SoftIntRegsFile 
*          0    00000ce0    00000000     DSECT

PieCtrlRegsFile 
*          0    00000ce0    0000001a     UNINITIALIZED
                  00000ce0    0000001a     F2837xD_GlobalVariableDefs.obj (PieCtrlRegsFile)

Cla1Prog   0    0000a000    00000200     
                  0000a000    000000d0     fcl_cla_code.obj (Cla1Prog:Cla1Task1)
                  0000a0d0    000000c4     fcl_cla_code.obj (Cla1Prog:Cla1Task4)
                  0000a194    0000002a     fcl_cla_code.obj (Cla1Prog:Cla1Task3)
                  0000a1be    00000022     fcl_cla_code.obj (Cla1Prog:Cla1Task2)
                  0000a1e0    00000008     fcl_f2837x_tmdxiddk_cla_tasks.obj (Cla1Prog:Cla1Task5)
                  0000a1e8    00000008     fcl_f2837x_tmdxiddk_cla_tasks.obj (Cla1Prog:Cla1Task6)
                  0000a1f0    00000008     fcl_f2837x_tmdxiddk_cla_tasks.obj (Cla1Prog:Cla1Task7)
                  0000a1f8    00000008     fcl_f2837x_tmdxiddk_cla_tasks.obj (Cla1Prog:Cla1Task8)

.text.1    0    0000d000    00001000     
                  0000d000    000006cc     PM_tformat_lib_f2837x.lib : pm_tformat_source.obj (.text)
                  0000d6cc    000005e0     fcl_f2837x_tmdxiddk.obj (.text:main)
                  0000dcac    000002b8     fcl_f2837x_tmdxiddk.obj (.text:buildLevel46)
                  0000df64    0000009c     rts2800_fpu32_eabi.lib : fd_add28.asm.obj (.text)

.text.2    0    0000e000    00001000     
                  0000e000    00000376     usblib_eabi.lib : usbhostenum.obj (.text:USBHostIntHandlerInternal)
                  0000e376    00000208     scistdio.obj (.text:SCIvprintf)
                  0000e57e    000001ff     usblib_eabi.lib : usbhostenum.obj (.text:USBHCDPipeAllocSize)
                  0000e77d    000001fa     sfra_f32_tmu_eabi.lib : sfra_f32_tmu_background.obj (.text)
                  0000e977    000001e0     sysctl.obj (.text:SysCtl_setClock)
                  0000eb57    000001dd     fcl_f2837x_tmdxiddk.obj (.text:readTformatEncPosition)
                  0000ed34    000001c2     sfra_f32_tmu_eabi.lib : sfra_f32_tmu_config_reset.obj (.text)
                  0000eef6    0000010a     usb_ex7_host_msc.obj (.text:ReadLine)

.text.3    0    0000f000    00001000     
                  0000f000    000001ad     usblib_eabi.lib : usbdconfig.obj (.text:USBDeviceConfig)
                  0000f1ad    0000016d     ff.obj (.text:auto_mount$20)
                  0000f31a    0000015c     sysctl.obj (.text:SysCtl_setAuxClock)
                  0000f476    00000156     usblib_eabi.lib : usbhostenum.obj (.text:ProcessUSBDeviceStateMachine)
                  0000f5cc    00000142     usb_ex7_host_msc.obj (.text:Cmd_cd)
                  0000f70e    00000136     ff.obj (.text:get_fileinfo$20)
                  0000f844    0000012f     rts2800_fpu32_eabi.lib : e_logf.c.obj (.text)
                  0000f973    0000012e     fcl_f2837x_tmdxiddk.obj (.text:configureGPIO)
                  0000faa1    0000012a     sfra_gui_scicomms_driverlib.obj (.text:SFRA_GUI_config)
                  0000fbcb    00000001     rts2800_fpu32_eabi.lib : _lock.c.obj (.text)
                  0000fbcc    0000012a     fcl_f2837x_tmdxiddk.obj (.text:configurePWM)
                  0000fcf6    00000127     usblib_eabi.lib : usbdenum.obj (.text:USBDGetDescriptor)
                  0000fe1d    00000126     sfra_gui_scicomms_driverlib.obj (.text:SFRA_GUI_sendData)
                  0000ff43    00000001     rts2800_fpu32_eabi.lib : startup.c.obj (.text)
                  0000ff44    000000b0     PM_tformat_lib_f2837x.lib : pm_tformat_crc.obj (.text)
                  0000fff4    0000000c     usblib_eabi.lib : usbdma.obj (.text:DMAUSBIntStatusClear)

.text.4    0    00010000    00001000     
                  00010000    00000126     usblib_eabi.lib : usbhostenum.obj (.text:USBHCDInitInternal)
                  00010126    00000115                     : usbhostenum.obj (.text:USBHCDPipeRead)
                  0001023b    00000100                     : usbdenum.obj (.text:USBDEP0StateTxConfig)
                  0001033b    00000100                     : usbhostenum.obj (.text:USBHCDPipeWrite)
                  0001043b    000000ff     usb_ex7_host_msc.obj (.text:USBMSCH_initUSB)
                  0001053a    000000f2     dio.obj (.text:DIO_init)
                  0001062c    000000f0     usblib_eabi.lib : usbhmsc.obj (.text:USBHMSCDriveReady)
                  0001071c    000000ee                     : usbhostenum.obj (.text:USBHCDPipeFree)
                  0001080a    000000ed                     : usbhhub.obj (.text:USBHHubMain)
                  000108f7    000000e7     fcl_f2837x_tmdxiddk.obj (.text:configurePIControllers)
                  000109de    000000e3     fcl_f2837x_tmdxiddk.obj (.text:configureADC)
                  00010ac1    000000e0     usb_ex7_host_msc.obj (.text:Cmd_ls)
                  00010ba1    000000de     device.obj (.text:Device_enableAllPeripherals)
                  00010c7f    000000de     rts2800_fpu32_eabi.lib : e_sqrt.c.obj (.text)
                  00010d5d    000000db     fcl_f2837x_tmdxiddk.obj (.text:configurePositionSensing)
                  00010e38    000000d9     ff.obj (.text:f_read)
                  00010f11    000000d0     usblib_eabi.lib : usbhostenum.obj (.text:USBHCDPipeConfig)
                  00010fe1    0000001f     usb_ex7_host_msc.obj (.text:Cmd_help)

.text.5    0    00011000    00001000     
                  00011000    000000ca     usblib_eabi.lib : usbdenum.obj (.text:USBDeviceEnumHandler)
                  000110ca    000000ca     driverlib_eabi.lib : usb.obj (.text:USBHostEndpointConfig)
                  00011194    000000c7     usblib_eabi.lib : usbhscsi.obj (.text:USBHSCSISendCommand)
                  0001125b    000000c6     usb_ex7_host_msc.obj (.text:Cmd_cat)
                  00011321    000000bf     usblib_eabi.lib : usbhostenum.obj (.text:USBHCDEnumHandler)
                  000113e0    000000af                     : usbdenum.obj (.text:USBDCDInit)
                  0001148f    000000ae                     : usbbuffer.obj (.text:HandleRxAvailable)
                  0001153d    000000ad     fcl_f2837x_tmdxiddk.obj (.text:A1)
                  000115ea    000000aa     fcl_f2837x_tmdxiddk.obj (.text:configureHVDMCProtection)
                  00011694    000000a6     usblib_eabi.lib : usbhostenum.obj (.text:USBHCDControlTransfer)
                  0001173a    0000009d                     : usbhostenum.obj (.text:USBHCDDeviceDisconnected)
                  000117d7    0000009b                     : usbdbulk.obj (.text:USBDBulkCompositeInit)
                  00011872    0000009a                     : usbdenum.obj (.text:USBDeviceIntHandlerInternal)
                  0001190c    00000097     fcl_f2837x_tmdxiddk.obj (.text:initFCLVars)
                  000119a3    00000095     usblib_eabi.lib : usbdenum.obj (.text:USBDSetInterface)
                  00011a38    00000090     ff.obj (.text:get_cluster$20)
                  00011ac8    0000008c     usblib_eabi.lib : usbhmsc.obj (.text:USBHMSCOpen)
                  00011b54    0000008b     adc.obj (.text:ADC_setMode)
                  00011bdf    0000008b     usblib_eabi.lib : usbhostenum.obj (.text:USBHostCheckPipes)
                  00011c6a    0000008a                     : usbbuffer.obj (.text:ScheduleNextTransmission)
                  00011cf4    00000089     driverlib_eabi.lib : usb.obj (.text:USBDevEndpointConfigSet)
                  00011d7d    00000089     ff.obj (.text:trace_path$20)
                  00011e06    00000088     usblib_eabi.lib : usbdenum.obj (.text:USBDClearFeature)
                  00011e8e    00000083                     : usbmode.obj (.text:USB0OTGModeIntHandler)
                  00011f11    00000083     fcl_f2837x_tmdxiddk.obj (.text:configureCLA)
                  00011f94    0000006c     usblib_eabi.lib : usbdenum.obj (.text:USBDGetStatus)

.text.6    0    00012022    00000fde     
                  00012022    00000083     rts2800_fpu32_eabi.lib : fd_mpy28.asm.obj (.text)
                  000120a5    00000082     usblib_eabi.lib : usbdma.obj (.text:USBLibDMAInit)
                  00012127    00000080                     : usbhostenum.obj (.text:FIFOAlloc)
                  000121a7    0000007d     fcl_f2837x_tmdxiddk.obj (.text:motorControlISR)
                  00012224    0000007c     usblib_eabi.lib : usbhostenum.obj (.text:USBHCDClearFeature)
                  000122a0    0000007b     ff.obj (.text:f_getfree)
                  0001231b    0000007b     ff.obj (.text:make_dirfile$20)
                  00012396    0000007a     interrupt.obj (.text:Interrupt_clearIFR)
                  00012410    00000079     usblib_eabi.lib : usbhostenum.obj (.text:USBHCDInit)
                  00012489    00000077     ff.obj (.text:f_open)
                  00012500    00000072     usblib_eabi.lib : usbhostenum.obj (.text:USBHCDOpenDriver)
                  00012572    00000071                     : usbdenum.obj (.text:USBDSetConfiguration)
                  000125e3    00000070                     : usbhostenum.obj (.text:USBHCDGetConfigDescriptor)
                  00012653    0000006e     driverlib_eabi.lib : usb.obj (.text:USBDevEndpointStallClear)
                  000126c1    0000006b     usblib_eabi.lib : usbdenum.obj (.text:USBDSetFeature)
                  0001272c    0000006b     driverlib_eabi.lib : usb.obj (.text:USBEndpointDataGet)
                  00012797    0000006a                        : usb.obj (.text:USBDevEndpointStatusClear)
                  00012801    0000006a     usblib_eabi.lib : usbhostenum.obj (.text:USBHCDHubDeviceConnected)
                  0001286b    00000069                     : usbdconfig.obj (.text:USBDeviceConfigAlternate)
                  000128d4    00000068                     : usbdenum.obj (.text:USBDEP0StateTx)
                  0001293c    00000068     fcl_tformat_f2837x_config.obj (.text:spiRxFIFOISR)
                  000129a4    00000067     sfra_f32_tmu_eabi.lib : sfra_f32_tmu_collect.obj (.text)
                  00012a0b    00000066     driverlib_eabi.lib : usb.obj (.text:USBFIFOConfigSet)
                  00012a71    00000064                        : usb.obj (.text:USBFIFOFlush)
                  00012ad5    00000063     dlog_4ch_f.obj (.text:DLOG_4CH_F_FUNC)
                  00012b38    00000063     usblib_eabi.lib : usbhostenum.obj (.text:USBHCDMain)
                  00012b9b    00000063     fcl_f2837x_sfra_gui.obj (.text:configureSFRA)
                  00012bfe    00000061     eeprom.obj (.text:EEPROM_init)
                  00012c5f    00000061     externflash.obj (.text:EXFLASH_init)
                  00012cc0    00000061     usb_ex4_dev_bulk.obj (.text:EchoNewDataToHost$23)
                  00012d21    0000005e     usblib_eabi.lib : usbdbulk.obj (.text:USBDBulkPacketRead)
                  00012d7f    0000005b                     : usbdbulk.obj (.text:USBDBulkInit)
                  00012dda    0000005b     driverlib_eabi.lib : usb.obj (.text:USBDevEndpointStall)
                  00012e35    0000005a     usblib_eabi.lib : usbhhub.obj (.text:HubDriverDeviceDisconnect)
                  00012e8f    00000059     clb.obj (.text:CLB_configCounterLoadMatch)
                  00012ee8    00000059     driverlib_eabi.lib : usb.obj (.text:USBEndpointDataSend)
                  00012f41    00000058     usblib_eabi.lib : usbdenum.obj (.text:USBDStringIndexFromRequest)
                  00012f99    00000058     driverlib_eabi.lib : usb.obj (.text:USBHostHubAddrSet)
                  00012ff1    0000000f     usblib_eabi.lib : usbbuffer.obj (.text:HandleTxComplete)

.text.7    0    00013000    00001000     
                  00013000    00000057     driverlib_eabi.lib : usb.obj (.text:USBIntStatus)
                  00013057    00000054                        : usb.obj (.text:USBEndpointDataPut)
                  000130ab    00000053     memcfg.obj (.text:MemCfg_getInitStatus)
                  000130fe    00000053     usblib_eabi.lib : usbringbuf.obj (.text:USBRingBufWrite)
                  00013151    00000052     memcfg.obj (.text:MemCfg_setLSRAMMasterSel)
                  000131a3    00000051     usblib_eabi.lib : usbhostenum.obj (.text:ConfigDescAlloc)
                  000131f4    00000051     ff.obj (.text:f_opendir)
                  00013245    0000004f     sfra_gui_scicomms_driverlib.obj (.text:SFRA_GUI_lifePulseTsk)
                  00013294    0000004f     usblib_eabi.lib : usbhscsi.obj (.text:USBHSCSIInquiry)
                  000132e3    0000004f     driverlib_eabi.lib : usb.obj (.text:USBHostEndpointStatusClear)
                  00013332    0000004e     usblib_eabi.lib : usbdbulk.obj (.text:ProcessDataFromHost)
                  00013380    0000004e                     : usbdbulk.obj (.text:USBDBulkPacketWrite)
                  000133ce    0000004e                     : usbdenum.obj (.text:USBDGetInterface)
                  0001341c    0000004d                     : usbhscsi.obj (.text:USBHSCSIReadCapacity)
                  00013469    0000004c                     : usbhscsi.obj (.text:USBHSCSIRequestSense)
                  000134b5    0000004c                     : usbhscsi.obj (.text:USBHSCSITestUnitReady)
                  00013501    0000004a                     : usbdenum.obj (.text:USBDReadAndDispatchRequest)
                  0001354b    0000004a     driverlib_eabi.lib : usb.obj (.text:USBDevEndpointDataAck)
                  00013595    00000049     usblib_eabi.lib : usbhostenum.obj (.text:USBHCDGetDeviceDescriptor)
                  000135de    00000048     interrupt.obj (.text:Interrupt_disable)
                  00013626    00000048     driverlib_eabi.lib : usb.obj (.text:_USBIndexWrite)
                  0001366e    00000048     fcl_f2837x_tmdxiddk.obj (.text:configureCMPSS)
                  000136b6    00000048     fcl_f2837x_tmdxiddk.obj (.text:configurePWM_1chUpCnt)
                  000136fe    00000048     ff.obj (.text:move_window$20)
                  00013746    00000047     driverlib_eabi.lib : usb.obj (.text:USBEndpointDataAvail)
                  0001378d    00000046     sysctl.obj (.text:SysCtl_getClock)
                  000137d3    00000044     usblib_eabi.lib : usbdcdesc.obj (.text:USBDCDConfigDescGet)
                  00013817    00000043     memcfg.obj (.text:MemCfg_initSections)
                  0001385a    00000043     usblib_eabi.lib : usbbuffer.obj (.text:USBBufferEventCallback)
                  0001389d    00000043     driverlib_eabi.lib : usb.obj (.text:USBHostEndpointDataAck)
                  000138e0    00000043     usblib_eabi.lib : usbringbuf.obj (.text:USBRingBufAdvanceWrite)
                  00013923    00000042     driverlib_eabi.lib : usb.obj (.text:USBHostAddrSet)
                  00013965    00000041     interrupt.obj (.text:Interrupt_initModule)
                  000139a6    00000040     driverlib_eabi.lib : usb.obj (.text:USBEndpointDataToggleClear)
                  000139e6    00000040                        : usb.obj (.text:USBHostRequestINClear)
                  00013a26    00000040     usblib_eabi.lib : usbmode.obj (.text:USBOTGSetMode)
                  00013a66    0000003f     gpio.obj (.text:GPIO_setPadConfig)
                  00013aa5    0000003f     driverlib_eabi.lib : usb.obj (.text:USBEndpointStatus)
                  00013ae4    0000003f                        : usb.obj (.text:USBHostRequestIN)
                  00013b23    0000003c     usblib_eabi.lib : usbhhub.obj (.text:HubGetPortStatus)
                  00013b5f    0000003b                     : usbdconfig.obj (.text:GetEPDescriptorType)
                  00013b9a    0000003b                     : usbdenum.obj (.text:USBDGetConfiguration)
                  00013bd5    0000003b                     : usbhostenum.obj (.text:USBHCDEP0StateTx)
                  00013c10    0000003b     driverlib_eabi.lib : usb.obj (.text:USBIntEnableControl)
                  00013c4b    0000003a     usblib_eabi.lib : usbmode.obj (.text:USB0DualModeIntHandler)
                  00013c85    00000039                     : usbdbulk.obj (.text:ProcessDataToHost)
                  00013cbe    00000039     driverlib_eabi.lib : usb.obj (.text:USBIntStatusControl)
                  00013cf7    00000037     usblib_eabi.lib : usbhhub.obj (.text:HubDriverReset)
                  00013d2e    00000037     sfra_gui_scicomms_driverlib.obj (.text:SFRA_GUI_getCmdByte)
                  00013d65    00000036     driverlib_eabi.lib : usb.obj (.text:USBHostPwrConfig)
                  00013d9b    00000035     usblib_eabi.lib : usbdbulk.obj (.text:HandleEndpoints)
                  00013dd0    00000035     usb_ex4_dev_bulk.obj (.text:RxHandler)
                  00013e05    00000035     ff.obj (.text:next_dir_entry$20)
                  00013e3a    00000034     usblib_eabi.lib : usbdbulk.obj (.text:HandleDevice)
                  00013e6e    00000034     interrupt.obj (.text:Interrupt_enable)
                  00013ea2    00000034     usblib_eabi.lib : usbbuffer.obj (.text:USBBufferInit)
                  00013ed6    00000034                     : usbhostenum.obj (.text:USBHCDPowerConfigSet)
                  00013f0a    00000034     ff.obj (.text:check_fs$20)
                  00013f3e    00000033     usblib_eabi.lib : usbhscsi.obj (.text:USBHSCSIRead10)
                  00013f71    00000032     sysctl.obj (.text:SysCtl_selectOscSource)
                  00013fa3    00000032     usblib_eabi.lib : usbhscsi.obj (.text:USBHSCSIWrite10)
                  00013fd5    0000002b                     : usbhostenum.obj (.text:ConfigDescFree)

.text.8    0    00014000    00001000     
                  00014000    00000031     usblib_eabi.lib : usbdcdesc.obj (.text:NextConfigDescGet)
                  00014031    00000031                     : usbdcdesc.obj (.text:USBDCDConfigGetInterfaceEndpoint)
                  00014062    00000031                     : usbdenum.obj (.text:USBDeviceEnumResetHandler)
                  00014093    00000031     rts2800_fpu32_eabi.lib : copy_decompress_lzss.c.obj (.text:decompress:lzss)
                  000140c4    00000031     usb_hal.obj (.text:f28x_USB0DeviceIntHandler)
                  000140f5    00000031     usb_hal.obj (.text:f28x_USB0DualModeIntHandler)
                  00014126    00000031     usb_hal.obj (.text:f28x_USB0HostIntHandler)
                  00014157    00000031     usb_hal.obj (.text:f28x_USB0OTGModeIntHandler)
                  00014188    00000030     gpio.obj (.text:GPIO_setPinConfig)
                  000141b8    00000030     usblib_eabi.lib : usbtick.obj (.text:InternalUSBRegisterTickHandler)
                  000141e8    0000002f                     : usbhostenum.obj (.text:USBHCDReset)
                  00014217    0000002e                     : usbdcdesc.obj (.text:ConfigAlternateInterfaceGet)
                  00014245    0000002e                     : usbdenum.obj (.text:USBDSetAddress)
                  00014273    0000002d                     : usbhostenum.obj (.text:USBHCDSetAddress)
                  000142a0    0000002d                     : usbhostenum.obj (.text:USBHCDSetConfig)
                  000142cd    0000002c     dlog_4ch_f.obj (.text:DLOG_4CH_F_init)
                  000142f9    0000002c     usblib_eabi.lib : usbhostenum.obj (.text:FIFOFree)
                  00014325    0000002c                     : usbdbulk.obj (.text:HandleConfigChange)
                  00014351    0000002c                     : usbhhub.obj (.text:HubClearPortFeature)
                  0001437d    0000002c                     : usbhhub.obj (.text:HubSetPortFeature)
                  000143a9    0000002c                     : usbdenum.obj (.text:USBDCDDeviceInfoInit)
                  000143d5    0000002c                     : usbdenum.obj (.text:USBDeviceResumeTickHandler)
                  00014401    0000002c                     : usbringbuf.obj (.text:USBRingBufInit)
                  0001442d    0000002b                     : usbdma.obj (.text:DMAUSBIntHandler)
                  00014458    0000002b                     : usbtick.obj (.text:InternalUSBStartOfFrameTick)
                  00014483    0000002b     sfra_gui_scicomms_driverlib.obj (.text:SFRA_GUI_getData)
                  000144ae    0000002b     usblib_eabi.lib : usbdesc.obj (.text:USBDescGet)
                  000144d9    0000002b                     : usbhmsc.obj (.text:USBHMSCBlockRead)
                  00014504    0000002b                     : usbhmsc.obj (.text:USBHMSCBlockWrite)
                  0001452f    0000002b     rts2800_fpu32_eabi.lib : autoinit.c.obj (.text:__TI_auto_init_nobinit_nopinit)
                  0001455a    0000002a     usblib_eabi.lib : usbdbulk.obj (.text:BulkTickHandler)
                  00014584    0000002a     sfra_gui_scicomms_driverlib.obj (.text:SFRA_GUI_echoCmdByte)
                  000145ae    0000002a     sfra_gui_scicomms_driverlib.obj (.text:SFRA_GUI_echoSizeByte)
                  000145d8    0000002a     rts2800_fpu32_eabi.lib : fd_cmp28.asm.obj (.text)
                  00014602    00000029     sfra_gui_scicomms_driverlib.obj (.text:SFRA_GUI_setData32)
                  0001462b    00000029     usb_ex4_dev_bulk.obj (.text:USBBD_initUSB)
                  00014654    00000029     usblib_eabi.lib : usbdesc.obj (.text:USBDescGetAlternateInterface)
                  0001467d    00000029                     : usbhmsc.obj (.text:USBHMSCGetMaxLUN)
                  000146a6    00000029     rts2800_fpu32_eabi.lib : exit.c.obj (.text)
                  000146cf    00000028     device.obj (.text:Device_enableUnbondedGPIOPullups)
                  000146f7    00000028     usblib_eabi.lib : usbbuffer.obj (.text:USBBufferInfoGet)
                  0001471f    00000028                     : usbdbulk.obj (.text:USBDBulkRxPacketAvailable)
                  00014747    00000027     device.obj (.text:Device_enableUnbondedGPIOPullupsFor100Pin)
                  0001476e    00000026     usblib_eabi.lib : usbdesc.obj (.text:USBDescGetNum)
                  00014794    00000026     sfra_f32_tmu_eabi.lib : sfra_f32_tmu_inject.obj (.text)
                  000147ba    00000025     usblib_eabi.lib : usbhhub.obj (.text:HubDriverDeviceConnect)
                  000147df    00000025                     : usbtick.obj (.text:InternalUSBTickInit)
                  00014804    00000025     sfra_gui_scicomms_driverlib.obj (.text:SFRA_GUI_echoDataByte)
                  00014829    00000025     usblib_eabi.lib : usbdcdesc.obj (.text:USBDCDConfigDescGetNum)
                  0001484e    00000025     usb_hal.obj (.text:USBGPIOEnable)
                  00014873    00000025     xbar.obj (.text:XBAR_setEPWMMuxConfig)
                  00014898    00000025     xbar.obj (.text:XBAR_setOutputMuxConfig)
                  000148bd    00000024     usblib_eabi.lib : usbdbulk.obj (.text:HandleDisconnect)
                  000148e1    00000024                     : usbringbuf.obj (.text:USBRingBufContigFree)
                  00014905    00000024     fat_usbmsc.obj (.text:disk_write)
                  00014929    00000023     fcl_cpu_code.obj (.text:FCL_initADC)
                  0001494c    00000023     rts2800_fpu32_eabi.lib : fd_tofsfpu32.asm.obj (.text)
                  0001496f    00000022     gpio.obj (.text:GPIO_setMasterCore)
                  00014991    00000022     gpio.obj (.text:GPIO_setQualificationMode)
                  000149b3    00000022     usblib_eabi.lib : usbdenum.obj (.text:SysCtl_resetPeripheral)
                  000149d5    00000022                     : usbhostenum.obj (.text:SysCtl_resetPeripheral)
                  000149f7    00000001     --HOLE-- [fill = 0]
                  000149f8    00000021     interrupt.obj (.text:Interrupt_initVectorTable)
                  00014a19    00000021     sci.obj (.text:SCI_setConfig)
                  00014a3a    00000021     driverlib_eabi.lib : usb.obj (.text:USBHostReset)
                  00014a5b    00000021                        : usb.obj (.text:USBHostResume)
                  00014a7c    00000021                        : usb.obj (.text:USBOTGSessionRequest)
                  00014a9d    00000021     usblib_eabi.lib : usbmode.obj (.text:USBStackModeSet)
                  00014abe    00000020     gpio.obj (.text:GPIO_setDirectionMode)
                  00014ade    00000020     sfra_gui_scicomms_driverlib.obj (.text:SFRA_GUI_cmdInterpreter)
                  00014afe    00000020     usblib_eabi.lib : usbhmsc.obj (.text:USBHMSCClose)
                  00014b1e    00000020                     : usbringbuf.obj (.text:USBRingBufAdvanceRead)
                  00014b3e    0000001f                     : usbbuffer.obj (.text:HandleRequestBuffer)
                  00014b5d    0000001f                     : usbhostenum.obj (.text:InternalUSBHCDSendEvent)
                  00014b7c    0000001f     spi.obj (.text:SPI_setConfig)
                  00014b9b    0000001f     usblib_eabi.lib : usbhostenum.obj (.text:USBHCDHubDeviceDisconnected)
                  00014bba    0000001f                     : usbmode.obj (.text:USBOTGRemovePower)
                  00014bd9    0000001e     device.obj (.text:Device_initGPIO)
                  00014bf7    0000001e     scistdio.obj (.text:SCIwrite)
                  00014c15    0000001e     spi.obj (.text:SPI_clearInterruptStatus)
                  00014c33    0000001d     device.obj (.text:Device_init)
                  00014c50    0000001d     sfra_gui_scicomms_driverlib.obj (.text:SFRA_GUI_getDataByte)
                  00014c6d    0000001d     sfra_gui_scicomms_driverlib.obj (.text:SFRA_GUI_getSizeByte)
                  00014c8a    0000001c     cla.obj (.text:CLA_setTriggerSource)
                  00014ca6    0000001c     usblib_eabi.lib : usbdconfig.obj (.text:GetEndpointFIFOSize)
                  00014cc2    0000001c     sci.obj (.text:SCI_clearInterruptStatus)
                  00014cde    0000001c     sfra_gui_scicomms_driverlib.obj (.text:SFRA_GUI_packWord)
                  00014cfa    0000001c     driverlib_eabi.lib : usb.obj (.text:USBIntEnableEndpoint)
                  00014d16    0000001c     fcl_f2837x_tmdxiddk.obj (.text:ramper)
                  00014d32    0000001c     rts2800_fpu32_eabi.lib : fs_tofdfpu32.asm.obj (.text)
                  00014d4e    0000001c                            : memcpy.c.obj (.text)
                  00014d6a    0000001b     fcl_f2837x_tmdxiddk.obj (.text:configureCMPSSFilter)
                  00014d85    0000001a     fcl_f2837x_tmdxiddk.obj (.text:A0)
                  00014d9f    0000001a     sci.obj (.text:SCI_enableInterrupt)
                  00014db9    0000001a     usblib_eabi.lib : usbbuffer.obj (.text:USBBufferDataWritten)
                  00014dd3    0000001a                     : usbdenum.obj (.text:USBDCDStallEP0)
                  00014ded    0000001a                     : usbdesc.obj (.text:USBDescGetInterface)
                  00014e07    0000001a     driverlib_eabi.lib : usb.obj (.text:USBEndpointDMADisable)
                  00014e21    0000001a     usblib_eabi.lib : usbringbuf.obj (.text:USBRingBufUsed)
                  00014e3b    0000001a                     : usbringbuf.obj (.text:UpdateIndexAtomic)
                  00014e55    00000019                     : usbdbulk.obj (.text:USBDBulkTxPacketAvailable)
                  00014e6e    00000019                     : usbdcdesc.obj (.text:USBDCDConfigDescGetSize)
                  00014e87    00000019                     : usbdcdesc.obj (.text:USBDCDConfigGetInterface)
                  00014ea0    00000019                     : usbringbuf.obj (.text:USBRingBufContigUsed)
                  00014eb9    00000018                     : usbdbulk.obj (.text:HandleResume)
                  00014ed1    00000018                     : usbdbulk.obj (.text:HandleSuspend)
                  00014ee9    00000018                     : usbhhub.obj (.text:HubDriverDeviceReset)
                  00014f01    00000018     spi.obj (.text:SPI_enableInterrupt)
                  00014f19    00000018     driverlib_eabi.lib : usb.obj (.text:USBIntStatusEndpoint)
                  00014f31    00000017     fcl_f2837x_tmdxiddk.obj (.text:B0)
                  00014f48    00000017     fcl_f2837x_tmdxiddk.obj (.text:C0)
                  00014f5f    00000017     fcl_cpu_code.obj (.text:FCL_initPWM)
                  00014f76    00000017     usblib_eabi.lib : usbdenum.obj (.text:SysCtl_enablePeripheral)
                  00014f8d    00000017                     : usbhostenum.obj (.text:SysCtl_enablePeripheral)
                  00014fa4    00000017     driverlib_eabi.lib : usb.obj (.text:USBDevDisconnect)
                  00014fbb    00000017                        : usb.obj (.text:USBDevMode)
                  00014fd2    00000017     usb_ex7_host_msc.obj (.text:USBHCDEvents)
                  00014fe9    00000017     driverlib_eabi.lib : usb.obj (.text:USBHostMode)

.text.9    0    00015000    000004aa     
                  00015000    00000017     driverlib_eabi.lib : usb.obj (.text:USBHostPwrDisable)
                  00015017    00000017                        : usb.obj (.text:USBHostPwrEnable)
                  0001502e    00000017                        : usb.obj (.text:USBHostRequestStatus)
                  00015045    00000017                        : usb.obj (.text:USBModeGet)
                  0001505c    00000017                        : usb.obj (.text:USBOTGMode)
                  00015073    00000017     fat_usbmsc.obj (.text:disk_read)
                  0001508a    00000017     rts2800_fpu32_eabi.lib : boot28.asm.obj (.text)
                  000150a1    00000016     cmpss.obj (.text:CMPSS_configFilterHigh)
                  000150b7    00000016     cmpss.obj (.text:CMPSS_configFilterLow)
                  000150cd    00000016     driverlib_eabi.lib : usb.obj (.text:USBDevConnect)
                  000150e3    00000016     usblib_eabi.lib : usbringbuf.obj (.text:USBRingBufFlush)
                  000150f9    00000016     ff.obj (.text:f_mount)
                  0001510f    00000016     fcl_f2837x_tmdxiddk.obj (.text:setupCpuTimer)
                  00015125    00000015     usblib_eabi.lib : usbbuffer.obj (.text:HandleDataRemaining)
                  0001513a    00000015     sysctl.obj (.text:SysCtl_getLowSpeedClock)
                  0001514f    00000015     usblib_eabi.lib : usbringbuf.obj (.text:USBRingBufFree)
                  00015164    00000015     ff.obj (.text:validate$20)
                  00015179    00000014     usblib_eabi.lib : usbhostenum.obj (.text:USBHCDRegisterDrivers)
                  0001518d    00000014     driverlib_eabi.lib : usb.obj (.text:USBHostSuspend)
                  000151a1    00000014     rts2800_fpu32_eabi.lib : strncpy.c.obj (.text)
                  000151b5    00000013     usb_ex7_host_msc.obj (.text:Cmd_pwd)
                  000151c8    00000013     gpio.obj (.text:GPIO_setAnalogMode)
                  000151db    00000013     usblib_eabi.lib : usbbuffer.obj (.text:USBBufferFlush)
                  000151ee    00000013                     : usbbuffer.obj (.text:USBBufferSpaceAvailable)
                  00015201    00000013     driverlib_eabi.lib : usb.obj (.text:USBDevAddrSet)
                  00015214    00000013     rts2800_fpu32_eabi.lib : memcmp.c.obj (.text)
                  00015227    00000012     usblib_eabi.lib : usbdbulk.obj (.text:SetDeferredOpFlag)
                  00015239    00000012                     : usbdhandler.obj (.text:USB0DeviceIntHandler)
                  0001524b    00000012                     : usbhostenum.obj (.text:USB0HostIntHandler)
                  0001525d    00000012                     : usbdesc.obj (.text:USBDescGetInterfaceEndpoint)
                  0001526f    00000012     fcl_f2837x_tmdxiddk.obj (.text:getVdc)
                  00015281    00000011     sfra_gui_scicomms_driverlib.obj (.text:SFRA_GUI_setButton)
                  00015292    00000011     sfra_gui_scicomms_driverlib.obj (.text:SFRA_GUI_setSlider)
                  000152a3    00000011     sfra_gui_scicomms_driverlib.obj (.text:SFRA_GUI_setText)
                  000152b4    00000011     usblib_eabi.lib : usbhostenum.obj (.text:USBHCDPowerConfigInit)
                  000152c5    00000011                     : usbhhub.obj (.text:USBHHubEnumerationComplete)
                  000152d6    00000011                     : usbhhub.obj (.text:USBHHubEnumerationError)
                  000152e7    00000011                     : usbhmsc.obj (.text:USBHMSCDriveOpen)
                  000152f8    00000011     driverlib_eabi.lib : usb.obj (.text:USBNumEndpointsGet)
                  00015309    00000010     fcl_f2837x_tmdxiddk.obj (.text:B1)
                  00015319    00000010     usb_ex7_host_msc.obj (.text:MSCCallback)
                  00015329    00000010     usblib_eabi.lib : usbmode.obj (.text:OTGDeviceDisconnect)
                  00015339    00000010                     : usbhostenum.obj (.text:SendUnknownConnect)
                  00015349    00000010                     : usbdenum.obj (.text:USBDSetDescriptor)
                  00015359    00000010                     : usbdenum.obj (.text:USBDSyncFrame)
                  00015369    00000010     ff.obj (.text:clust2sect$20)
                  00015379    0000000f     sfra_gui_scicomms_driverlib.obj (.text:SFRA_GUI_runSerialHostComms)
                  00015388    0000000e     rts2800_fpu32_eabi.lib : fd_sub28.asm.obj (.text)
                  00015396    0000000d     fcl_f2837x_tmdxiddk.obj (.text:C1)
                  000153a3    0000000d     usblib_eabi.lib : usbringbuf.obj (.text:Interrupt_disableMaster)
                  000153b0    0000000d                     : usbringbuf.obj (.text:Interrupt_enableMaster)
                  000153bd    0000000d                     : usbhhub.obj (.text:USBHHubInit)
                  000153ca    0000000c     usb_ex4_dev_bulk.obj (.text:TxHandler)
                  000153d6    0000000c     rts2800_fpu32_eabi.lib : args_main.c.obj (.text)
                  000153e2    0000000b     usblib_eabi.lib : usbhostenum.obj (.text:USBHCDPowerAutomatic)
                  000153ed    0000000a     rts2800_fpu32_eabi.lib : strcmp.c.obj (.text)
                  000153f7    00000008                            : copy_decompress_none.c.obj (.text:decompress:none)
                  000153ff    00000008                            : strcat.c.obj (.text)
                  00015407    00000008     fcl_tformat_f2837x_config.obj (.text:tformat_checkCRC)
                  0001540f    00000007     scistdio.obj (.text:SCIprintf)
                  00015416    00000007     usblib_eabi.lib : usbdma.obj (.text:uDMAUSBChannelAllocate)
                  0001541d    00000007                     : usbdma.obj (.text:uDMAUSBChannelStatus)
                  00015424    00000007                     : usbdma.obj (.text:uDMAUSBTransfer)
                  0001542b    00000006     fcl_f2837x_tmdxiddk.obj (.text:A2)
                  00015431    00000006     fcl_f2837x_tmdxiddk.obj (.text:A3)
                  00015437    00000006     fcl_f2837x_tmdxiddk.obj (.text:B2)
                  0001543d    00000006     fcl_f2837x_tmdxiddk.obj (.text:B3)
                  00015443    00000006     fcl_f2837x_tmdxiddk.obj (.text:C2)
                  00015449    00000006     fcl_f2837x_tmdxiddk.obj (.text:C3)
                  0001544f    00000006     cputimer.obj (.text:CPUTimer_setEmulationMode)
                  00015455    00000006     rts2800_fpu32_eabi.lib : copy_zero_init.c.obj (.text:decompress:ZI)
                  0001545b    00000006                            : memset.c.obj (.text)
                  00015461    00000005     usblib_eabi.lib : usbdma.obj (.text:DMAUSBStatus)
                  00015466    00000005     sfra_gui_scicomms_driverlib.obj (.text:SFRA_GUI_spareTsk08)
                  0001546b    00000005     usblib_eabi.lib : usbdma.obj (.text:uDMAUSBArbSizeSet)
                  00015470    00000005                     : usbdma.obj (.text:uDMAUSBChannelDisable)
                  00015475    00000005                     : usbdma.obj (.text:uDMAUSBChannelEnable)
                  0001547a    00000005                     : usbdma.obj (.text:uDMAUSBChannelIntDisable)
                  0001547f    00000005                     : usbdma.obj (.text:uDMAUSBChannelIntEnable)
                  00015484    00000005                     : usbdma.obj (.text:uDMAUSBChannelRelease)
                  00015489    00000005                     : usbdma.obj (.text:uDMAUSBIntStatus)
                  0001548e    00000005                     : usbdma.obj (.text:uDMAUSBUnitSizeSet)
                  00015493    00000004     fcl_cpu_code.obj (.text:FCL_initQEP)
                  00015497    00000004     interrupt.obj (.text:Interrupt_defaultHandler)
                  0001549b    00000004     usb_ex4_dev_bulk.obj (.text:ModeCallback)
                  0001549f    00000003     device.obj (.text:__error__)
                  000154a2    00000002     fcl_cpu_code.obj (.text:FCL_getSwVersion)
                  000154a4    00000002     interrupt.obj (.text:Interrupt_illegalOperationHandler)
                  000154a6    00000002     interrupt.obj (.text:Interrupt_nmiHandler)
                  000154a8    00000002     rts2800_fpu32_eabi.lib : pre_init.c.obj (.text)

.TI.ramfunc 
*          0    000154aa    00000220     
                  000154aa    0000011e     fcl_cpu_code.obj (.TI.ramfunc:FCL_runPICtrl)
                  000155c8    000000c5     fcl_cpu_code.obj (.TI.ramfunc:FCL_runPICtrlWrap)
                  0001568d    00000039     fcl_cpu_code.obj (.TI.ramfunc:FCL_resetController)
                  000156c6    00000004     sysctl.obj (.TI.ramfunc)

MODULE SUMMARY

       Module                                   code    ro data   rw data
       ------                                   ----    -------   -------
    .\common\
       sysctl.obj                               973     0         0      
       device.obj                               363     0         6      
       interrupt.obj                            352     0         0      
       memcfg.obj                               232     0         0      
       gpio.obj                                 230     0         0      
       adc.obj                                  139     0         0      
       clb.obj                                  89      0         0      
       sci.obj                                  87      0         0      
       spi.obj                                  85      0         0      
       xbar.obj                                 74      0         0      
       cmpss.obj                                44      0         0      
       cla.obj                                  28      0         0      
       F2837xD_GlobalVariableDefs.obj           0       0         26     
       cputimer.obj                             6       0         0      
       F2837xD_CodeStartBranch.obj              2       0         0      
    +--+----------------------------------------+-------+---------+---------+
       Total:                                   2704    0         32     
                                                                         
    .\sources\
       fcl_f2837x_tmdxiddk.obj                  5080    12        2040   
       usb_ex7_host_msc.obj                     1354    12        1562   
       ff.obj                                   1855    0         5      
       sfra_gui_scicomms_driverlib.obj          1120    0         264    
       fcl_cpu_code.obj                         604     0         478    
       fcl_f2837x_sfra_gui.obj                  99      0         732    
       usb_ex4_dev_bulk_structs.obj             0       198       612    
       scistdio.obj                             557     0         2      
       fcl_cla_code.obj                         480     0         16     
       fcl_tformat_f2837x_config.obj            112     0         342    
       dio.obj                                  242     0         0      
       usb_hal.obj                              233     0         0      
       usb_ex4_dev_bulk.obj                     207     0         12     
       dlog_4ch_f.obj                           143     0         0      
       eeprom.obj                               97      0         0      
       externflash.obj                          97      0         0      
       fat_usbmsc.obj                           59      0         1      
       fcl_f2837x_tmdxiddk_cla_tasks.obj        32      0         0      
       cmdline.obj                              0       0         18     
    +--+----------------------------------------+-------+---------+---------+
       Total:                                   12371   222       6084   
                                                                         
    C:\Users\WAYNE~1.CHI\AppData\Local\Temp\
       {DA63AF40-C2BB-4A41-BBFD-0095D79A7F7D}   0       1062      0      
    +--+----------------------------------------+-------+---------+---------+
       Total:                                   0       1062      0      
                                                                         
    C:/Users/wayne.chiang/Downloads/git/c2000ware_motorcontrol/libraries/position_sensing/tformat/lib/PM_tformat_lib_f2837x.lib
       pm_tformat_source.obj                    1740    0         32     
       pm_tformat_crc.obj                       176     0         0      
    +--+----------------------------------------+-------+---------+---------+
       Total:                                   1916    0         32     
                                                                         
    C:\Users\wayne.chiang\Downloads\git\c2000ware_motorcontrol\c2000ware\driverlib\f2837xd\driverlib\ccs\Debug\driverlib_eabi.lib
       usb.obj                                  2595    96        0      
    +--+----------------------------------------+-------+---------+---------+
       Total:                                   2595    96        0      
                                                                         
    C:\Users\wayne.chiang\Downloads\git\c2000ware_motorcontrol\c2000ware\libraries\communications\usb\f2837xd\lib\usblib_eabi.lib
       usbhostenum.obj                          5159    125       894    
       usbdenum.obj                             2396    150       118    
       usbdbulk.obj                             911     185       31     
       usbdconfig.obj                           621     126       0      
       usbbuffer.obj                            602     118       0      
       usbhhub.obj                              638     0         62     
       usbhscsi.obj                             608     0         0      
       usbhmsc.obj                              556     8         14     
       usbringbuf.obj                           408     119       0      
       usbdma.obj                               251     115       140    
       usbmode.obj                              333     116       10     
       usbdcdesc.obj                            299     0         0      
       usbdesc.obj                              166     0         0      
       usbtick.obj                              128     0         30     
       usbdhandler.obj                          18      0         0      
    +--+----------------------------------------+-------+---------+---------+
       Total:                                   13094   1062      1299   
                                                                         
    C:\Users\wayne.chiang\Downloads\git\c2000ware_motorcontrol\libraries\sfra\lib\sfra_f32_tmu_eabi.lib
       sfra_f32_tmu_background.obj              506     0         0      
       sfra_f32_tmu_config_reset.obj            450     0         34     
       sfra_f32_tmu_collect.obj                 103     0         0      
       sfra_f32_tmu_inject.obj                  38      0         0      
    +--+----------------------------------------+-------+---------+---------+
       Total:                                   1097    0         34     
                                                                         
    C:\ti\ccs920\ccs\tools\compiler\ti-cgt-c2000_18.12.3.LTS\lib\rts2800_fpu32_eabi.lib
       e_logf.c.obj                             303     0         0      
       e_sqrt.c.obj                             222     0         0      
       fd_add28.asm.obj                         156     0         0      
       fd_mpy28.asm.obj                         131     0         0      
       copy_decompress_lzss.c.obj               49      0         0      
       exit.c.obj                               41      0         6      
       autoinit.c.obj                           43      0         0      
       fd_cmp28.asm.obj                         42      0         0      
       fd_tofsfpu32.asm.obj                     35      0         0      
       fs_tofdfpu32.asm.obj                     28      0         0      
       memcpy.c.obj                             28      0         0      
       boot28.asm.obj                           23      0         0      
       strncpy.c.obj                            20      0         0      
       memcmp.c.obj                             19      0         0      
       fd_sub28.asm.obj                         14      0         0      
       args_main.c.obj                          12      0         0      
       strcmp.c.obj                             10      0         0      
       copy_decompress_none.c.obj               8       0         0      
       strcat.c.obj                             8       0         0      
       copy_zero_init.c.obj                     6       0         0      
       memset.c.obj                             6       0         0      
       _lock.c.obj                              1       0         2      
       pre_init.c.obj                           2       0         0      
       errno.c.obj                              0       0         1      
       startup.c.obj                            1       0         0      
    +--+----------------------------------------+-------+---------+---------+
       Total:                                   1208    0         9      
                                                                         
       Stack:                                   0       0         896    
       Linker Generated:                        0       334       0      
    +--+----------------------------------------+-------+---------+---------+
       Grand Total:                             34985   2776      8386   


LINKER GENERATED COPY TABLES

__TI_cinit_table @ 0000893c records: 5, size/record: 4, table size: 20
	.data: load addr=00008800, load size=00000124 bytes, run addr=0001a000, run size=00000d9d bytes, compression=lzss
	.bss: load addr=0000892a, load size=00000004 bytes, run addr=00019000, run size=00000f20 bytes, compression=zero_init
	.bss_cla: load addr=0000892e, load size=00000004 bytes, run addr=00009100, run size=00000010 bytes, compression=zero_init
	ClaData: load addr=00008932, load size=00000004 bytes, run addr=00009800, run size=0000003a bytes, compression=zero_init
	SFRA_F32_Data: load addr=00008936, load size=00000004 bytes, run addr=00012000, run size=00000022 bytes, compression=zero_init


LINKER GENERATED HANDLER TABLE

__TI_handler_table @ 00008924 records: 3, size/record: 2, table size: 6
	index: 0, handler: __TI_zero_init
	index: 1, handler: __TI_decompress_lzss
	index: 2, handler: __TI_decompress_none


GLOBAL DATA SYMBOLS: SORTED BY DATA PAGE

address     data page           name
--------    ----------------    ----
00000400      10 (00000400)     __stack

00000ce0      33 (00000cc0)     PieCtrlRegs

00009100     244 (00009100)     Q_cla
0000910e     244 (00009100)     ClaQep

00009800     260 (00009800)     lsw
00009802     260 (00009800)     pangle
00009804     260 (00009800)     speedWe
00009806     260 (00009800)     rg1
00009812     260 (00009800)     qep1
00009824     260 (00009800)     pi_iq

00012000     480 (00012000)     _SFRA_F32_state
00012001     480 (00012000)     _SFRA_F32_stateSlew
00012002     480 (00012000)     _SFRA_F32_rSinSum
00012004     480 (00012000)     _SFRA_F32_rCosSum
00012006     480 (00012000)     _SFRA_F32_uSinSum
00012008     480 (00012000)     _SFRA_F32_uCosSum
0001200a     480 (00012000)     _SFRA_F32_ySinSum
0001200c     480 (00012000)     _SFRA_F32_yCosSum
0001200e     480 (00012000)     _SFRA_F32_pointerStart
00012010     480 (00012000)     _SFRA_F32_reference
00012012     480 (00012000)     _SFRA_F32_amplitude
00012014     480 (00012000)     _SFRA_F32_scalar
00012016     480 (00012000)     _SFRA_F32_step
00012018     480 (00012000)     _SFRA_F32_pointer
0001201a     480 (00012000)     _SFRA_F32_preCount
0001201c     480 (00012000)     _SFRA_F32_count
0001201e     480 (00012000)     _SFRA_F32_windowSamples
00012020     480 (00012000)     _SFRA_F32_angle

00019000     640 (00019000)     g_eState
00019001     640 (00019000)     g_eUIState

0001944a     651 (00019440)     g_pui8USBRxBuffer

0001954a     655 (00019540)     g_pui8USBTxBuffer

0001964a     659 (00019640)     tformatCRCtable

0001974a     65d (00019740)     g_psDCDInst

00019780     65e (00019780)     speedWePrev
00019782     65e (00019780)     curA_PPBRESULT
00019784     65e (00019780)     curB_PPBRESULT
00019786     65e (00019780)     curC_PPBRESULT
00019788     65e (00019780)     voltDC_PPBRESULT
0001978a     65e (00019780)     AdcIntFlag
0001978c     65e (00019780)     pwmCompA
0001978e     65e (00019780)     pwmCompB
00019790     65e (00019780)     pwmCompC
00019792     65e (00019780)     clarke1
0001979c     65e (00019780)     park1
000197aa     65e (00019780)     D_cpu

000197c0     65f (000197c0)     svgen1
000197d2     65f (000197c0)     pi_id

00019800     660 (00019800)     FCL_params

000198aa     662 (00019880)     g_pHCDPool

0001992a     664 (00019900)     clMagVect

0001998e     666 (00019980)     clPhaseVect

000199f2     667 (000199c0)     freqVect

00019a56     669 (00019a40)     olMagVect

00019aba     66a (00019a80)     olPhaseVect

00019b1e     66c (00019b00)     plantMagVect

00019b82     66e (00019b80)     plantPhaseVect

00019bf8     66f (00019bc0)     SFRA_GUI_cmdPacket
00019bfe     66f (00019bc0)     g_ppsDevInfo

00019c00     670 (00019c00)     tFormat_dataId
00019c02     670 (00019c00)     Alpha_State_Ptr
00019c04     670 (00019c00)     A_Task_Ptr
00019c06     670 (00019c00)     B_Task_Ptr
00019c08     670 (00019c00)     C_Task_Ptr
00019c0a     670 (00019c00)     offset_SDFM1
00019c0c     670 (00019c00)     offset_SDFM2
00019c0e     670 (00019c00)     tformatAngle
00019c10     670 (00019c00)     tformatSpd
00019c12     670 (00019c00)     retVal1
00019c14     670 (00019c00)     crcResult
00019c16     670 (00019c00)     position
00019c18     670 (00019c00)     turns
00019c1a     670 (00019c00)     speed1

00019c40     671 (00019c40)     dlog_4ch1
00019c5a     671 (00019c40)     SFRA_GUI_commsOKflg
00019c5b     671 (00019c40)     SFRA_GUI_serialCommsTimer
00019c5c     671 (00019c40)     SFRA_GUI_lowByteFlag
00019c5d     671 (00019c40)     SFRA_GUI_sendTaskPtr
00019c5e     671 (00019c40)     SFRA_GUI_rxChar
00019c5f     671 (00019c40)     SFRA_GUI_rxWord
00019c60     671 (00019c40)     SFRA_GUI_taskDoneFlag
00019c61     671 (00019c40)     SFRA_GUI_numWords
00019c62     671 (00019c40)     SFRA_GUI_wordsLeftToGet
00019c63     671 (00019c40)     SFRA_GUI_dataOut16
00019c64     671 (00019c40)     SFRA_GUI_rcvTskPtrShdw
00019c65     671 (00019c40)     SFRA_GUI_delayer
00019c66     671 (00019c40)     SFRA_GUI_memGetPtr
00019c67     671 (00019c40)     SFRA_GUI_memGetAmount
00019c68     671 (00019c40)     SFRA_GUI_memSetPtr
00019c69     671 (00019c40)     SFRA_GUI_led_flag
00019c6a     671 (00019c40)     SFRA_GUI_led_gpio
00019c6b     671 (00019c40)     SFRA_GUI_sweep_start
00019c6c     671 (00019c40)     SFRA_GUI_rcvTaskPointer
00019c6e     671 (00019c40)     SFRA_GUI_sci_base_addr
00019c70     671 (00019c40)     SFRA_GUI_dataOut32
00019c72     671 (00019c40)     SFRA_GUI_memDataPtr16
00019c74     671 (00019c40)     SFRA_GUI_memDataPtr32
00019c76     671 (00019c40)     SFRA_GUI_memGetAddress
00019c78     671 (00019c40)     SFRA_GUI_memSetValue
00019c7a     671 (00019c40)     SFRA_GUI_temp

00019c80     672 (00019c80)     tformatData

00019da6     676 (00019d80)     g_pfnTickHandlers

00019dfe     677 (00019dc0)     SFRA_GUI_arrayGetList

00019e1e     678 (00019e00)     SFRA_GUI_cmdDispatcher
00019e3e     678 (00019e00)     SFRA_GUI_dataSetList

00019e5e     679 (00019e40)     SFRA_GUI_varGetList
00019e7e     679 (00019e40)     SFRA_GUI_varSetBtnList

00019e9e     67a (00019e80)     SFRA_GUI_varSetSldrList
00019ebe     67a (00019e80)     SFRA_GUI_varSetTxtList

00019ede     67b (00019ec0)     sfra1

00019f0a     67c (00019f00)     g_pvTickInstance
00019f16     67c (00019f00)     g_eOTGModeState
00019f18     67c (00019f00)     g_ui32PollRate
00019f1c     67c (00019f00)     g_eCurrentUSBMode
00019f1e     67c (00019f00)     g_pcStatus

0001a362     68d (0001a340)     DBUFF_4CH1

0001a4f2     693 (0001a4c0)     DBUFF_4CH2

0001a682     69a (0001a680)     DBUFF_4CH3

0001a812     6a0 (0001a800)     DBUFF_4CH4

0001a9a2     6a6 (0001a980)     g_pui8BulkDeviceDescriptor
0001a9b4     6a6 (0001a980)     g_pui8BulkDescriptor
0001a9be     6a6 (0001a980)     _lock

0001a9c0     6a7 (0001a9c0)     serialCommsTimer
0001a9c1     6a7 (0001a9c0)     offsetCalCounter
0001a9c2     6a7 (0001a9c0)     hlt
0001a9c3     6a7 (0001a9c0)     llt
0001a9c4     6a7 (0001a9c0)     clkPrescale
0001a9c5     6a7 (0001a9c0)     sampWin
0001a9c6     6a7 (0001a9c0)     thresh
0001a9c7     6a7 (0001a9c0)     LEM_curHi
0001a9c8     6a7 (0001a9c0)     LEM_curLo
0001a9c9     6a7 (0001a9c0)     SHUNT_curHi
0001a9ca     6a7 (0001a9c0)     SHUNT_curLo
0001a9cb     6a7 (0001a9c0)     enableFlag
0001a9cc     6a7 (0001a9c0)     backTicker
0001a9cd     6a7 (0001a9c0)     tripFlagDMC
0001a9ce     6a7 (0001a9c0)     clearTripFlagDMC
0001a9cf     6a7 (0001a9c0)     runMotor
0001a9d0     6a7 (0001a9c0)     ledCnt1
0001a9d1     6a7 (0001a9c0)     speedLoopPrescaler
0001a9d2     6a7 (0001a9c0)     speedLoopCount
0001a9d3     6a7 (0001a9c0)     lsw2EntryFlag
0001a9d4     6a7 (0001a9c0)     FCL_cycleCount
0001a9d5     6a7 (0001a9c0)     fclClrCntr
0001a9d6     6a7 (0001a9c0)     fclCycleCountMax
0001a9d7     6a7 (0001a9c0)     posPtrMax
0001a9d8     6a7 (0001a9c0)     posPtr
0001a9d9     6a7 (0001a9c0)     sfraTestLoop
0001a9da     6a7 (0001a9c0)     tFormat_encCmdStatus
0001a9db     6a7 (0001a9c0)     tFormat_crcError
0001a9dc     6a7 (0001a9c0)     offset_lemV
0001a9de     6a7 (0001a9c0)     offset_lemW
0001a9e0     6a7 (0001a9c0)     offset_lemU
0001a9e2     6a7 (0001a9c0)     offset_IP
0001a9e4     6a7 (0001a9c0)     offset_DcImcu
0001a9e6     6a7 (0001a9c0)     K1
0001a9e8     6a7 (0001a9c0)     K2
0001a9ea     6a7 (0001a9c0)     curLimit
0001a9ec     6a7 (0001a9c0)     isrTicker
0001a9ee     6a7 (0001a9c0)     fclLatencyInMicroSec
0001a9f0     6a7 (0001a9c0)     maxModIndex
0001a9f2     6a7 (0001a9c0)     T
0001a9f4     6a7 (0001a9c0)     VdTesting
0001a9f6     6a7 (0001a9c0)     VqTesting
0001a9f8     6a7 (0001a9c0)     IdRef
0001a9fa     6a7 (0001a9c0)     tempIdRef
0001a9fc     6a7 (0001a9c0)     IqRef
0001a9fe     6a7 (0001a9c0)     speedRef

0001aa00     6a8 (0001aa00)     lsw1Speed
0001aa02     6a8 (0001aa00)     alignCntr
0001aa04     6a8 (0001aa00)     alignCnt
0001aa06     6a8 (0001aa00)     alignInitCnt
0001aa08     6a8 (0001aa00)     IdRef_start
0001aa0a     6a8 (0001aa00)     IdRef_run
0001aa0c     6a8 (0001aa00)     posCntr
0001aa0e     6a8 (0001aa00)     posCntrMax
0001aa10     6a8 (0001aa00)     posSlewRate
0001aa12     6a8 (0001aa00)     dlogCh1
0001aa14     6a8 (0001aa00)     dlogCh2
0001aa16     6a8 (0001aa00)     dlogCh3
0001aa18     6a8 (0001aa00)     dlogCh4
0001aa1a     6a8 (0001aa00)     sfraCollectStart
0001aa1c     6a8 (0001aa00)     sfraNoiseD
0001aa1e     6a8 (0001aa00)     sfraNoiseQ
0001aa20     6a8 (0001aa00)     sfraNoiseW
0001aa22     6a8 (0001aa00)     angMax
0001aa24     6a8 (0001aa00)     ipark1

0001aa40     6a9 (0001aa40)     rc1
0001aa50     6a9 (0001aa40)     tFormat
0001aa60     6a9 (0001aa40)     pi_pos

0001aa80     6aa (0001aa80)     spdObs
0001aa9a     6aa (0001aa80)     pid_pos

0001aac0     6ab (0001aac0)     pid_spd
0001aae8     6ab (0001aac0)     posEncElecTheta
0001aaf6     6ab (0001aac0)     adcHandle

0001ab00     6ac (0001ab00)     cm1_const
0001ab10     6ac (0001ab00)     cm1
0001ab24     6ac (0001ab00)     volt1

0001ab40     6ad (0001ab40)     se1_const
0001ab58     6ad (0001ab40)     se1

0001ab80     6ae (0001ab80)     fe1_const

0001abc0     6af (0001abc0)     fe1

0001ac06     6b0 (0001ac00)     g_sFresultStrings
0001ac3e     6b0 (0001ac00)     g_psMSCInstance

0001ac40     6b1 (0001ac40)     g_sTxBuffer
0001ac5c     6b1 (0001ac40)     g_sRxBuffer

0001ac80     6b2 (0001ac80)     g_sBulkDevice

0001acf4     6b3 (0001acc0)     g_psCmdTable

0001ad2a     6b4 (0001ad00)     tformat_tile1HLCInstr

0001ad4a     6b5 (0001ad40)     posEncMechTheta
0001ad68     6b5 (0001ad40)     g_ui32TxCount
0001ad6a     6b5 (0001ad40)     g_ui32RxCount
0001ad6c     6b5 (0001ad40)     g_ui32Flags
0001ad6e     6b5 (0001ad40)     Example_Result
0001ad70     6b5 (0001ad40)     Example_PassCount
0001ad72     6b5 (0001ad40)     Example_Fail
0001ad74     6b5 (0001ad40)     pwmHandle
0001ad7a     6b5 (0001ad40)     __TI_enable_exit_profile_output
0001ad7c     6b5 (0001ad40)     __TI_cleanup_ptr
0001ad7e     6b5 (0001ad40)     __TI_dtors_ptr

0001ad80     6b6 (0001ad80)     g_bUSBTimerInitialized
0001ad82     6b6 (0001ad80)     g_ui32CurrentUSBTick
0001ad84     6b6 (0001ad80)     g_ui32USBSOFCount
0001ad86     6b6 (0001ad80)     g_psBulkSections
0001ad8a     6b6 (0001ad80)     g_iUSBMode
0001ad8c     6b6 (0001ad80)     g_ui32WaitTicks
0001ad8e     6b6 (0001ad80)     vTimer0
0001ad92     6b6 (0001ad80)     vTimer1
0001ad96     6b6 (0001ad80)     vTimer2
0001ad9c     6b6 (0001ad80)     errno

0001b844     6e1 (0001b840)     g_pui8ConfigString
0001b874     6e1 (0001b840)     g_pui8DataInterfaceString

0001b89c     6e2 (0001b880)     g_pui8ProductString

0001b8c4     6e3 (0001b8c0)     g_pui8ManufacturerString
0001b8e8     6e3 (0001b8c0)     g_pui8BulkInterface

0001b900     6e4 (0001b900)     g_sBulkConfigSection
0001b904     6e4 (0001b900)     g_sBulkInterfaceSection
0001b908     6e4 (0001b900)     g_sBulkConfigHeader
0001b90c     6e4 (0001b900)     g_sBulkHandlers
0001b93e     6e4 (0001b900)     g_pui8SerialNumberString

0001b95c     6e5 (0001b940)     g_ppui8StringDescriptors
0001b974     6e5 (0001b940)     g_sUSBEventDriver

0001b980     6e6 (0001b980)     g_sUSBHostMSCClassDriver
0001b988     6e6 (0001b980)     g_pui8LangDescriptor
0001b98c     6e6 (0001b980)     g_ppBulkConfigDescriptors


GLOBAL SYMBOLS: SORTED ALPHABETICALLY BY Name 

page  address   name                                     
----  -------   ----                                     
0     00014d85  A0                                       
0     0001153d  A1                                       
0     0001542b  A2                                       
0     00015431  A3                                       
0     00011b54  ADC_setMode                              
0     00019c04  A_Task_Ptr                               
0     0001978a  AdcIntFlag                               
0     00019c02  Alpha_State_Ptr                          
0     00014f31  B0                                       
0     00015309  B1                                       
0     00015437  B2                                       
0     0001543d  B3                                       
0     00019c06  B_Task_Ptr                               
0     000146a6  C$$EXIT                                  
0     00014f48  C0                                       
0     00015396  C1                                       
0     00015443  C2                                       
0     00015449  C3                                       
abs   00000100  CLA_SCRATCHPAD_SIZE                      
0     00014c8a  CLA_setTriggerSource                     
0     00012e8f  CLB_configCounterLoadMatch               
0     000150a1  CMPSS_configFilterHigh                   
0     000150b7  CMPSS_configFilterLow                    
0     0001544f  CPUTimer_setEmulationMode                
0     00019c08  C_Task_Ptr                               
0     0000a000  Cla1Task1                                
0     0000a1be  Cla1Task2                                
0     0000a194  Cla1Task3                                
0     0000a0d0  Cla1Task4                                
0     0000a1e0  Cla1Task5                                
0     0000a1e8  Cla1Task6                                
0     0000a1f0  Cla1Task7                                
0     0000a1f8  Cla1Task8                                
0     0000910e  ClaQep                                   
0     0001125b  Cmd_cat                                  
0     0000f5cc  Cmd_cd                                   
0     00010fe1  Cmd_help                                 
0     00010ac1  Cmd_ls                                   
0     000151b5  Cmd_pwd                                  
0     000131a3  ConfigDescAlloc                          
0     00013fd5  ConfigDescFree                           
0     0001a362  DBUFF_4CH1                               
0     0001a4f2  DBUFF_4CH2                               
0     0001a682  DBUFF_4CH3                               
0     0001a812  DBUFF_4CH4                               
0     0001053a  DIO_init                                 
0     00012ad5  DLOG_4CH_F_FUNC                          
0     000142cd  DLOG_4CH_F_init                          
0     000197aa  D_cpu                                    
0     00010ba1  Device_enableAllPeripherals              
0     000146cf  Device_enableUnbondedGPIOPullups         
0     00014747  Device_enableUnbondedGPIOPullupsFor100Pin
0     00014c33  Device_init                              
0     00014bd9  Device_initGPIO                          
0     00012bfe  EEPROM_init                              
0     00012c5f  EXFLASH_init                             
0     0001ad72  Example_Fail                             
0     0001ad70  Example_PassCount                        
0     0001ad6e  Example_Result                           
0     0001a9d4  FCL_cycleCount                           
0     000154a2  FCL_getSwVersion                         
0     00014929  FCL_initADC                              
0     00014f5f  FCL_initPWM                              
0     00015493  FCL_initQEP                              
0     00019800  FCL_params                               
0     0001568d  FCL_resetController                      
0     000154aa  FCL_runPICtrl                            
0     000155c8  FCL_runPICtrlWrap                        
0     000151c8  GPIO_setAnalogMode                       
0     00014abe  GPIO_setDirectionMode                    
0     0001496f  GPIO_setMasterCore                       
0     00013a66  GPIO_setPadConfig                        
0     00014188  GPIO_setPinConfig                        
0     00014991  GPIO_setQualificationMode                
0     0001a9f8  IdRef                                    
0     0001aa0a  IdRef_run                                
0     0001aa08  IdRef_start                              
0     00014b5d  InternalUSBHCDSendEvent                  
0     000141b8  InternalUSBRegisterTickHandler           
0     00014458  InternalUSBStartOfFrameTick              
0     000147df  InternalUSBTickInit                      
0     000135de  Interrupt_disable                        
0     00013e6e  Interrupt_enable                         
0     00013965  Interrupt_initModule                     
0     000149f8  Interrupt_initVectorTable                
0     0001a9fc  IqRef                                    
0     0001a9e6  K1                                       
0     0001a9e8  K2                                       
0     0001a9c7  LEM_curHi                                
0     0001a9c8  LEM_curLo                                
0     00015319  MSCCallback                              
0     000130ab  MemCfg_getInitStatus                     
0     00013817  MemCfg_initSections                      
0     00013151  MemCfg_setLSRAMMasterSel                 
0     0001549b  ModeCallback                             
0     00015329  OTGDeviceDisconnect                      
0     0000ff97  PM_tformat_generateCRCTable              
0     0000ff44  PM_tformat_getCRC                        
0     0000d5a8  PM_tformat_receiveData                   
0     0000d581  PM_tformat_setFreq                       
0     0000d397  PM_tformat_setupCommand                  
0     0000d2ec  PM_tformat_setupPeriph                   
0     0000d2d7  PM_tformat_startOperation                
0     00000ce0  PieCtrlRegs                              
0     00009100  Q_cla                                    
0     0000eef6  ReadLine                                 
0     00013dd0  RxHandler                                
0     00014cc2  SCI_clearInterruptStatus                 
0     00014d9f  SCI_enableInterrupt                      
0     00014a19  SCI_setConfig                            
0     0001540f  SCIprintf                                
0     0000e376  SCIvprintf                               
0     00014bf7  SCIwrite                                 
0     0000ee98  SFRA_F32_config                          
0     0000ee6e  SFRA_F32_initFreqArrayWithLogSteps       
0     0000ee45  SFRA_F32_reset                           
0     0000ed3c  SFRA_F32_resetFreqRespArray              
0     0000e77d  SFRA_F32_runBackgroundTask               
0     0000ed34  SFRA_F32_updateInjectionAmplitude        
0     00019dfe  SFRA_GUI_arrayGetList                    
0     00019e1e  SFRA_GUI_cmdDispatcher                   
0     00014ade  SFRA_GUI_cmdInterpreter                  
0     00019bf8  SFRA_GUI_cmdPacket                       
0     00019c5a  SFRA_GUI_commsOKflg                      
0     0000faa1  SFRA_GUI_config                          
0     00019c63  SFRA_GUI_dataOut16                       
0     00019c70  SFRA_GUI_dataOut32                       
0     00019e3e  SFRA_GUI_dataSetList                     
0     00019c65  SFRA_GUI_delayer                         
0     00014584  SFRA_GUI_echoCmdByte                     
0     00014804  SFRA_GUI_echoDataByte                    
0     000145ae  SFRA_GUI_echoSizeByte                    
0     0000fe1d  SFRA_GUI_getArray                        
0     00013d2e  SFRA_GUI_getCmdByte                      
0     00014483  SFRA_GUI_getData                         
0     00014c50  SFRA_GUI_getDataByte                     
0     00014c6d  SFRA_GUI_getSizeByte                     
0     0000fe1d  SFRA_GUI_getVariable                     
0     00019c69  SFRA_GUI_led_flag                        
0     00019c6a  SFRA_GUI_led_gpio                        
0     00013245  SFRA_GUI_lifePulseTsk                    
0     00019c5c  SFRA_GUI_lowByteFlag                     
0     00019c72  SFRA_GUI_memDataPtr16                    
0     00019c74  SFRA_GUI_memDataPtr32                    
0     00019c76  SFRA_GUI_memGetAddress                   
0     00019c67  SFRA_GUI_memGetAmount                    
0     00019c66  SFRA_GUI_memGetPtr                       
0     00019c68  SFRA_GUI_memSetPtr                       
0     00019c78  SFRA_GUI_memSetValue                     
0     00019c61  SFRA_GUI_numWords                        
0     00014cde  SFRA_GUI_packWord                        
0     00019c6c  SFRA_GUI_rcvTaskPointer                  
0     00019c64  SFRA_GUI_rcvTskPtrShdw                   
0     00015379  SFRA_GUI_runSerialHostComms              
0     00019c5e  SFRA_GUI_rxChar                          
0     00019c5f  SFRA_GUI_rxWord                          
0     00019c6e  SFRA_GUI_sci_base_addr                   
0     0000fe1d  SFRA_GUI_sendData                        
0     00019c5d  SFRA_GUI_sendTaskPtr                     
0     00019c5b  SFRA_GUI_serialCommsTimer                
0     00015281  SFRA_GUI_setButton                       
0     00014602  SFRA_GUI_setData32                       
0     00015292  SFRA_GUI_setSlider                       
0     000152a3  SFRA_GUI_setText                         
0     00015466  SFRA_GUI_spareTsk08                      
0     00019c6b  SFRA_GUI_sweep_start                     
0     00019c60  SFRA_GUI_taskDoneFlag                    
0     00019c7a  SFRA_GUI_temp                            
0     00019e5e  SFRA_GUI_varGetList                      
0     00019e7e  SFRA_GUI_varSetBtnList                   
0     00019e9e  SFRA_GUI_varSetSldrList                  
0     00019ebe  SFRA_GUI_varSetTxtList                   
0     00019c62  SFRA_GUI_wordsLeftToGet                  
0     0001a9c9  SHUNT_curHi                              
0     0001a9ca  SHUNT_curLo                              
0     00014c15  SPI_clearInterruptStatus                 
0     00014f01  SPI_enableInterrupt                      
0     00014b7c  SPI_setConfig                            
0     000156c6  SysCtl_delay                             
0     0001378d  SysCtl_getClock                          
0     0001513a  SysCtl_getLowSpeedClock                  
0     00013f71  SysCtl_selectOscSource                   
0     0000f31a  SysCtl_setAuxClock                       
0     0000e977  SysCtl_setClock                          
0     0001a9f2  T                                        
0     000153ca  TxHandler                                
0     00015239  USB0DeviceIntHandler                     
0     00013c4b  USB0DualModeIntHandler                   
0     0001524b  USB0HostIntHandler                       
0     00011e8e  USB0OTGModeIntHandler                    
0     0001462b  USBBD_initUSB                            
0     00014db9  USBBufferDataWritten                     
0     0001385a  USBBufferEventCallback                   
0     000151db  USBBufferFlush                           
0     000146f7  USBBufferInfoGet                         
0     00013ea2  USBBufferInit                            
0     000151ee  USBBufferSpaceAvailable                  
0     000117d7  USBDBulkCompositeInit                    
0     00012d7f  USBDBulkInit                             
0     00012d21  USBDBulkPacketRead                       
0     00013380  USBDBulkPacketWrite                      
0     0001471f  USBDBulkRxPacketAvailable                
0     00014e55  USBDBulkTxPacketAvailable                
0     000137d3  USBDCDConfigDescGet                      
0     00014829  USBDCDConfigDescGetNum                   
0     00014e6e  USBDCDConfigDescGetSize                  
0     00014e87  USBDCDConfigGetInterface                 
0     00014031  USBDCDConfigGetInterfaceEndpoint         
0     000143a9  USBDCDDeviceInfoInit                     
0     000113e0  USBDCDInit                               
0     00014dd3  USBDCDStallEP0                           
0     000144ae  USBDescGet                               
0     00014ded  USBDescGetInterface                      
0     0001525d  USBDescGetInterfaceEndpoint              
0     0001476e  USBDescGetNum                            
0     00015201  USBDevAddrSet                            
0     000150cd  USBDevConnect                            
0     00014fa4  USBDevDisconnect                         
0     00011cf4  USBDevEndpointConfigSet                  
0     0001354b  USBDevEndpointDataAck                    
0     00012dda  USBDevEndpointStall                      
0     00012653  USBDevEndpointStallClear                 
0     00012797  USBDevEndpointStatusClear                
0     00014fbb  USBDevMode                               
0     0000f000  USBDeviceConfig                          
0     0001286b  USBDeviceConfigAlternate                 
0     00011000  USBDeviceEnumHandler                     
0     00014062  USBDeviceEnumResetHandler                
0     00011872  USBDeviceIntHandlerInternal              
0     000143d5  USBDeviceResumeTickHandler               
0     00014e07  USBEndpointDMADisable                    
0     00013746  USBEndpointDataAvail                     
0     0001272c  USBEndpointDataGet                       
0     00013057  USBEndpointDataPut                       
0     00012ee8  USBEndpointDataSend                      
0     000139a6  USBEndpointDataToggleClear               
0     00013aa5  USBEndpointStatus                        
0     00012a0b  USBFIFOConfigSet                         
0     00012a71  USBFIFOFlush                             
0     0001484e  USBGPIOEnable                            
0     00011694  USBHCDControlTransfer                    
0     00014fd2  USBHCDEvents                             
0     00012801  USBHCDHubDeviceConnected                 
0     00014b9b  USBHCDHubDeviceDisconnected              
0     00012410  USBHCDInit                               
0     00012b38  USBHCDMain                               
0     0000e57e  USBHCDPipeAllocSize                      
0     00010f11  USBHCDPipeConfig                         
0     0001071c  USBHCDPipeFree                           
0     00010126  USBHCDPipeRead                           
0     0001033b  USBHCDPipeWrite                          
0     000153e2  USBHCDPowerAutomatic                     
0     000152b4  USBHCDPowerConfigInit                    
0     00013ed6  USBHCDPowerConfigSet                     
0     00015179  USBHCDRegisterDrivers                    
0     000141e8  USBHCDReset                              
0     00014273  USBHCDSetAddress                         
0     000142a0  USBHCDSetConfig                          
0     000152c5  USBHHubEnumerationComplete               
0     000152d6  USBHHubEnumerationError                  
0     000153bd  USBHHubInit                              
0     0001080a  USBHHubMain                              
0     000144d9  USBHMSCBlockRead                         
0     00014504  USBHMSCBlockWrite                        
0     000152e7  USBHMSCDriveOpen                         
0     0001062c  USBHMSCDriveReady                        
0     00013294  USBHSCSIInquiry                          
0     00013f3e  USBHSCSIRead10                           
0     0001341c  USBHSCSIReadCapacity                     
0     00013469  USBHSCSIRequestSense                     
0     000134b5  USBHSCSITestUnitReady                    
0     00013fa3  USBHSCSIWrite10                          
0     00013923  USBHostAddrSet                           
0     00011bdf  USBHostCheckPipes                        
0     000110ca  USBHostEndpointConfig                    
0     0001389d  USBHostEndpointDataAck                   
0     000132e3  USBHostEndpointStatusClear               
0     00012f99  USBHostHubAddrSet                        
0     0000e000  USBHostIntHandlerInternal                
0     00014fe9  USBHostMode                              
0     00013d65  USBHostPwrConfig                         
0     00015000  USBHostPwrDisable                        
0     00015017  USBHostPwrEnable                         
0     00013ae4  USBHostRequestIN                         
0     000139e6  USBHostRequestINClear                    
0     0001502e  USBHostRequestStatus                     
0     00014a3a  USBHostReset                             
0     00014a5b  USBHostResume                            
0     0001518d  USBHostSuspend                           
0     00013c10  USBIntEnableControl                      
0     00014cfa  USBIntEnableEndpoint                     
0     00013000  USBIntStatus                             
0     00013cbe  USBIntStatusControl                      
0     00014f19  USBIntStatusEndpoint                     
0     000120a5  USBLibDMAInit                            
0     0001043b  USBMSCH_initUSB                          
0     00015045  USBModeGet                               
0     000152f8  USBNumEndpointsGet                       
0     0001505c  USBOTGMode                               
0     00014a7c  USBOTGSessionRequest                     
0     00014b1e  USBRingBufAdvanceRead                    
0     000138e0  USBRingBufAdvanceWrite                   
0     000148e1  USBRingBufContigFree                     
0     00014ea0  USBRingBufContigUsed                     
0     000150e3  USBRingBufFlush                          
0     0001514f  USBRingBufFree                           
0     00014401  USBRingBufInit                           
0     00014e21  USBRingBufUsed                           
0     000130fe  USBRingBufWrite                          
0     00014a9d  USBStackModeSet                          
0     0001a9f4  VdTesting                                
0     0001a9f6  VqTesting                                
0     00014873  XBAR_setEPWMMuxConfig                    
0     00014898  XBAR_setOutputMuxConfig                  
0     00012012  _SFRA_F32_amplitude                      
0     00012020  _SFRA_F32_angle                          
0     0001201c  _SFRA_F32_count                          
0     00012018  _SFRA_F32_pointer                        
0     0001200e  _SFRA_F32_pointerStart                   
0     0001201a  _SFRA_F32_preCount                       
0     00012004  _SFRA_F32_rCosSum                        
0     00012002  _SFRA_F32_rSinSum                        
0     00012010  _SFRA_F32_reference                      
0     00012014  _SFRA_F32_scalar                         
0     00012000  _SFRA_F32_state                          
0     00012001  _SFRA_F32_stateSlew                      
0     00012016  _SFRA_F32_step                           
0     00012008  _SFRA_F32_uCosSum                        
0     00012006  _SFRA_F32_uSinSum                        
0     0001201e  _SFRA_F32_windowSamples                  
0     0001200c  _SFRA_F32_yCosSum                        
0     0001200a  _SFRA_F32_ySinSum                        
0     000129a4  __SFRA_F32_collect                       
0     00014794  __SFRA_F32_inject                        
0     0000893c  __TI_CINIT_Base                          
0     00008950  __TI_CINIT_Limit                         
0     00008924  __TI_Handler_Table_Base                  
0     0000892a  __TI_Handler_Table_Limit                 
0     00000780  __TI_STACK_END                           
abs   00000380  __TI_STACK_SIZE                          
0     0001452f  __TI_auto_init_nobinit_nopinit           
0     0001ad7c  __TI_cleanup_ptr                         
0     00014093  __TI_decompress_lzss                     
0     000153f7  __TI_decompress_none                     
0     0001ad7e  __TI_dtors_ptr                           
0     0001ad7a  __TI_enable_exit_profile_output          
abs   ffffffff  __TI_pprof_out_hndl                      
abs   ffffffff  __TI_prof_data_size                      
abs   ffffffff  __TI_prof_data_start                     
0     00015455  __TI_zero_init                           
0     0000df64  __c28xabi_addd                           
0     000145d8  __c28xabi_cmpd                           
0     0001494c  __c28xabi_dtof                           
0     00014d32  __c28xabi_ftod                           
0     00012022  __c28xabi_mpyd                           
0     00015388  __c28xabi_subd                           
n/a   UNDEFED   __c_args__                               
0     0001549f  __error__                                
0     00000400  __stack                                  
0     000153d6  _args_main                               
0     0001508a  _c_int00                                 
0     0001a9be  _lock                                    
0     0000fbcb  _nop                                     
0     0000ff43  _system_post_cinit                       
0     000154a8  _system_pre_init                         
0     000146a6  abort                                    
0     0001aaf6  adcHandle                                
0     0001aa04  alignCnt                                 
0     0001aa02  alignCntr                                
0     0001aa06  alignInitCnt                             
0     0001aa22  angMax                                   
0     0001a9cc  backTicker                               
0     0001992a  clMagVect                                
0     0001998e  clPhaseVect                              
0     00019792  clarke1                                  
0     0001a9ce  clearTripFlagDMC                         
0     0001a9c4  clkPrescale                              
0     0001ab10  cm1                                      
0     0001ab00  cm1_const                                
0     00000000  code_start                               
0     000109de  configureADC                             
0     00011f11  configureCLA                             
0     0001366e  configureCMPSS                           
0     00014d6a  configureCMPSSFilter                     
0     0000f973  configureGPIO                            
0     000115ea  configureHVDMCProtection                 
0     000108f7  configurePIControllers                   
0     0000fbcc  configurePWM                             
0     000136b6  configurePWM_1chUpCnt                    
0     00010d5d  configurePositionSensing                 
0     00012b9b  configureSFRA                            
0     00019c14  crcResult                                
0     00019782  curA_PPBRESULT                           
0     00019784  curB_PPBRESULT                           
0     00019786  curC_PPBRESULT                           
0     0001a9ea  curLimit                                 
0     00015073  disk_read                                
0     00014905  disk_write                               
0     0001aa12  dlogCh1                                  
0     0001aa14  dlogCh2                                  
0     0001aa16  dlogCh3                                  
0     0001aa18  dlogCh4                                  
0     00019c40  dlog_4ch1                                
0     0001a9cb  enableFlag                               
0     0001ad9c  errno                                    
0     000146a8  exit                                     
0     000140c4  f28x_USB0DeviceIntHandler                
0     000140f5  f28x_USB0DualModeIntHandler              
0     00014126  f28x_USB0HostIntHandler                  
0     00014157  f28x_USB0OTGModeIntHandler               
0     000122a0  f_getfree                                
0     000150f9  f_mount                                  
0     00012489  f_open                                   
0     000131f4  f_opendir                                
0     00010e38  f_read                                   
0     0001a9d5  fclClrCntr                               
0     0001a9d6  fclCycleCountMax                         
0     0001a9ee  fclLatencyInMicroSec                     
0     0001abc0  fe1                                      
0     0001ab80  fe1_const                                
0     000199f2  freqVect                                 
0     0001ad80  g_bUSBTimerInitialized                   
0     00019f1c  g_eCurrentUSBMode                        
0     00019f16  g_eOTGModeState                          
0     00019000  g_eState                                 
0     00019001  g_eUIState                               
0     0001ad8a  g_iUSBMode                               
0     000198aa  g_pHCDPool                               
0     00019f1e  g_pcStatus                               
0     00019da6  g_pfnTickHandlers                        
0     0001b98c  g_ppBulkConfigDescriptors                
0     00019bfe  g_ppsDevInfo                             
0     0001b95c  g_ppui8StringDescriptors                 
0     0001ad86  g_psBulkSections                         
0     0001acf4  g_psCmdTable                             
0     0001974a  g_psDCDInst                              
0     0001ac3e  g_psMSCInstance                          
0     0001a9b4  g_pui8BulkDescriptor                     
0     0001a9a2  g_pui8BulkDeviceDescriptor               
0     0001b8e8  g_pui8BulkInterface                      
0     0001b844  g_pui8ConfigString                       
0     0001b874  g_pui8DataInterfaceString                
0     0001b988  g_pui8LangDescriptor                     
0     0001b8c4  g_pui8ManufacturerString                 
0     0001b89c  g_pui8ProductString                      
0     0001b93e  g_pui8SerialNumberString                 
0     0001944a  g_pui8USBRxBuffer                        
0     0001954a  g_pui8USBTxBuffer                        
0     00019f0a  g_pvTickInstance                         
0     0001b908  g_sBulkConfigHeader                      
0     0001b900  g_sBulkConfigSection                     
0     0001ac80  g_sBulkDevice                            
0     0001b90c  g_sBulkHandlers                          
0     0001b904  g_sBulkInterfaceSection                  
0     0001ac06  g_sFresultStrings                        
0     0001ac5c  g_sRxBuffer                              
0     0001ac40  g_sTxBuffer                              
0     0001b974  g_sUSBEventDriver                        
0     0001b980  g_sUSBHostMSCClassDriver                 
0     0001ad82  g_ui32CurrentUSBTick                     
0     0001ad6c  g_ui32Flags                              
0     00019f18  g_ui32PollRate                           
0     0001ad6a  g_ui32RxCount                            
0     0001ad68  g_ui32TxCount                            
0     0001ad84  g_ui32USBSOFCount                        
0     0001ad8c  g_ui32WaitTicks                          
0     0001a9c2  hlt                                      
0     0001190c  initFCLVars                              
0     0001aa24  ipark1                                   
0     0001a9ec  isrTicker                                
0     0001a9d0  ledCnt1                                  
0     0001a9c3  llt                                      
0     0000f844  logf                                     
0     00009800  lsw                                      
0     0001aa00  lsw1Speed                                
0     0001a9d3  lsw2EntryFlag                            
0     0000d6cc  main                                     
0     0001a9f0  maxModIndex                              
0     00015214  memcmp                                   
0     00014d4e  memcpy                                   
0     0001545b  memset                                   
0     000121a7  motorControlISR                          
0     0001a9c1  offsetCalCounter                         
0     0001a9e4  offset_DcImcu                            
0     0001a9e2  offset_IP                                
0     00019c0a  offset_SDFM1                             
0     00019c0c  offset_SDFM2                             
0     0001a9e0  offset_lemU                              
0     0001a9dc  offset_lemV                              
0     0001a9de  offset_lemW                              
0     00019a56  olMagVect                                
0     00019aba  olPhaseVect                              
0     00009802  pangle                                   
0     0001979c  park1                                    
0     000197d2  pi_id                                    
0     00009824  pi_iq                                    
0     0001aa60  pi_pos                                   
0     0001aa9a  pid_pos                                  
0     0001aac0  pid_spd                                  
0     00019b1e  plantMagVect                             
0     00019b82  plantPhaseVect                           
0     0001aa0c  posCntr                                  
0     0001aa0e  posCntrMax                               
0     0001aae8  posEncElecTheta                          
0     0001ad4a  posEncMechTheta                          
0     0001a9d8  posPtr                                   
0     0001a9d7  posPtrMax                                
0     0001aa10  posSlewRate                              
0     00019c16  position                                 
0     0001978c  pwmCompA                                 
0     0001978e  pwmCompB                                 
0     00019790  pwmCompC                                 
0     0001ad74  pwmHandle                                
0     00009812  qep1                                     
0     00014d16  ramper                                   
0     0001aa40  rc1                                      
0     0000eb57  readTformatEncPosition                   
0     00019c12  retVal1                                  
0     00009806  rg1                                      
0     0001a9cf  runMotor                                 
0     0001a9c5  sampWin                                  
0     0001ab58  se1                                      
0     0001ab40  se1_const                                
0     0001a9c0  serialCommsTimer                         
0     0001510f  setupCpuTimer                            
0     00019ede  sfra1                                    
0     0001aa1a  sfraCollectStart                         
0     0001aa1c  sfraNoiseD                               
0     0001aa1e  sfraNoiseQ                               
0     0001aa20  sfraNoiseW                               
0     0001a9d9  sfraTestLoop                             
0     0001aa80  spdObs                                   
0     00019c1a  speed1                                   
0     0001a9d2  speedLoopCount                           
0     0001a9d1  speedLoopPrescaler                       
0     0001a9fe  speedRef                                 
0     00009804  speedWe                                  
0     00019780  speedWePrev                              
0     0001293c  spiRxFIFOISR                             
0     00010c7f  sqrt                                     
0     00010c7f  sqrtl                                    
0     000153ff  strcat                                   
0     000153ed  strcmp                                   
0     000151a1  strncpy                                  
0     000197c0  svgen1                                   
0     0001aa50  tFormat                                  
0     0001a9db  tFormat_crcError                         
0     00019c00  tFormat_dataId                           
0     0001a9da  tFormat_encCmdStatus                     
0     0001a9fa  tempIdRef                                
0     00019c0e  tformatAngle                             
0     0001964a  tformatCRCtable                          
0     00019c80  tformatData                              
0     00019c10  tformatSpd                               
0     00015407  tformat_checkCRC                         
0     0000d29e  tformat_configureSPILen                  
0     0000d1f1  tformat_getBits                          
0     0000d101  tformat_initCLB4                         
0     0000d100  tformat_initCLBXBAR                      
0     0000d098  tformat_initSPIFIFO                      
0     0000d039  tformat_putBits                          
0     0000d000  tformat_resetCLB                         
0     0001ad2a  tformat_tile1HLCInstr                    
0     0001a9c6  thresh                                   
0     0001a9cd  tripFlagDMC                              
0     00019c18  turns                                    
0     0001ad8e  vTimer0                                  
0     0001ad92  vTimer1                                  
0     0001ad96  vTimer2                                  
0     0001ab24  volt1                                    
0     00019788  voltDC_PPBRESULT                         


GLOBAL SYMBOLS: SORTED BY Symbol Address 

page  address   name                                     
----  -------   ----                                     
0     00000000  code_start                               
0     00000400  __stack                                  
0     00000780  __TI_STACK_END                           
0     00000ce0  PieCtrlRegs                              
0     00008924  __TI_Handler_Table_Base                  
0     0000892a  __TI_Handler_Table_Limit                 
0     0000893c  __TI_CINIT_Base                          
0     00008950  __TI_CINIT_Limit                         
0     00009100  Q_cla                                    
0     0000910e  ClaQep                                   
0     00009800  lsw                                      
0     00009802  pangle                                   
0     00009804  speedWe                                  
0     00009806  rg1                                      
0     00009812  qep1                                     
0     00009824  pi_iq                                    
0     0000a000  Cla1Task1                                
0     0000a0d0  Cla1Task4                                
0     0000a194  Cla1Task3                                
0     0000a1be  Cla1Task2                                
0     0000a1e0  Cla1Task5                                
0     0000a1e8  Cla1Task6                                
0     0000a1f0  Cla1Task7                                
0     0000a1f8  Cla1Task8                                
0     0000d000  tformat_resetCLB                         
0     0000d039  tformat_putBits                          
0     0000d098  tformat_initSPIFIFO                      
0     0000d100  tformat_initCLBXBAR                      
0     0000d101  tformat_initCLB4                         
0     0000d1f1  tformat_getBits                          
0     0000d29e  tformat_configureSPILen                  
0     0000d2d7  PM_tformat_startOperation                
0     0000d2ec  PM_tformat_setupPeriph                   
0     0000d397  PM_tformat_setupCommand                  
0     0000d581  PM_tformat_setFreq                       
0     0000d5a8  PM_tformat_receiveData                   
0     0000d6cc  main                                     
0     0000df64  __c28xabi_addd                           
0     0000e000  USBHostIntHandlerInternal                
0     0000e376  SCIvprintf                               
0     0000e57e  USBHCDPipeAllocSize                      
0     0000e77d  SFRA_F32_runBackgroundTask               
0     0000e977  SysCtl_setClock                          
0     0000eb57  readTformatEncPosition                   
0     0000ed34  SFRA_F32_updateInjectionAmplitude        
0     0000ed3c  SFRA_F32_resetFreqRespArray              
0     0000ee45  SFRA_F32_reset                           
0     0000ee6e  SFRA_F32_initFreqArrayWithLogSteps       
0     0000ee98  SFRA_F32_config                          
0     0000eef6  ReadLine                                 
0     0000f000  USBDeviceConfig                          
0     0000f31a  SysCtl_setAuxClock                       
0     0000f5cc  Cmd_cd                                   
0     0000f844  logf                                     
0     0000f973  configureGPIO                            
0     0000faa1  SFRA_GUI_config                          
0     0000fbcb  _nop                                     
0     0000fbcc  configurePWM                             
0     0000fe1d  SFRA_GUI_getArray                        
0     0000fe1d  SFRA_GUI_getVariable                     
0     0000fe1d  SFRA_GUI_sendData                        
0     0000ff43  _system_post_cinit                       
0     0000ff44  PM_tformat_getCRC                        
0     0000ff97  PM_tformat_generateCRCTable              
0     00010126  USBHCDPipeRead                           
0     0001033b  USBHCDPipeWrite                          
0     0001043b  USBMSCH_initUSB                          
0     0001053a  DIO_init                                 
0     0001062c  USBHMSCDriveReady                        
0     0001071c  USBHCDPipeFree                           
0     0001080a  USBHHubMain                              
0     000108f7  configurePIControllers                   
0     000109de  configureADC                             
0     00010ac1  Cmd_ls                                   
0     00010ba1  Device_enableAllPeripherals              
0     00010c7f  sqrt                                     
0     00010c7f  sqrtl                                    
0     00010d5d  configurePositionSensing                 
0     00010e38  f_read                                   
0     00010f11  USBHCDPipeConfig                         
0     00010fe1  Cmd_help                                 
0     00011000  USBDeviceEnumHandler                     
0     000110ca  USBHostEndpointConfig                    
0     0001125b  Cmd_cat                                  
0     000113e0  USBDCDInit                               
0     0001153d  A1                                       
0     000115ea  configureHVDMCProtection                 
0     00011694  USBHCDControlTransfer                    
0     000117d7  USBDBulkCompositeInit                    
0     00011872  USBDeviceIntHandlerInternal              
0     0001190c  initFCLVars                              
0     00011b54  ADC_setMode                              
0     00011bdf  USBHostCheckPipes                        
0     00011cf4  USBDevEndpointConfigSet                  
0     00011e8e  USB0OTGModeIntHandler                    
0     00011f11  configureCLA                             
0     00012000  _SFRA_F32_state                          
0     00012001  _SFRA_F32_stateSlew                      
0     00012002  _SFRA_F32_rSinSum                        
0     00012004  _SFRA_F32_rCosSum                        
0     00012006  _SFRA_F32_uSinSum                        
0     00012008  _SFRA_F32_uCosSum                        
0     0001200a  _SFRA_F32_ySinSum                        
0     0001200c  _SFRA_F32_yCosSum                        
0     0001200e  _SFRA_F32_pointerStart                   
0     00012010  _SFRA_F32_reference                      
0     00012012  _SFRA_F32_amplitude                      
0     00012014  _SFRA_F32_scalar                         
0     00012016  _SFRA_F32_step                           
0     00012018  _SFRA_F32_pointer                        
0     0001201a  _SFRA_F32_preCount                       
0     0001201c  _SFRA_F32_count                          
0     0001201e  _SFRA_F32_windowSamples                  
0     00012020  _SFRA_F32_angle                          
0     00012022  __c28xabi_mpyd                           
0     000120a5  USBLibDMAInit                            
0     000121a7  motorControlISR                          
0     000122a0  f_getfree                                
0     00012410  USBHCDInit                               
0     00012489  f_open                                   
0     00012653  USBDevEndpointStallClear                 
0     0001272c  USBEndpointDataGet                       
0     00012797  USBDevEndpointStatusClear                
0     00012801  USBHCDHubDeviceConnected                 
0     0001286b  USBDeviceConfigAlternate                 
0     0001293c  spiRxFIFOISR                             
0     000129a4  __SFRA_F32_collect                       
0     00012a0b  USBFIFOConfigSet                         
0     00012a71  USBFIFOFlush                             
0     00012ad5  DLOG_4CH_F_FUNC                          
0     00012b38  USBHCDMain                               
0     00012b9b  configureSFRA                            
0     00012bfe  EEPROM_init                              
0     00012c5f  EXFLASH_init                             
0     00012d21  USBDBulkPacketRead                       
0     00012d7f  USBDBulkInit                             
0     00012dda  USBDevEndpointStall                      
0     00012e8f  CLB_configCounterLoadMatch               
0     00012ee8  USBEndpointDataSend                      
0     00012f99  USBHostHubAddrSet                        
0     00013000  USBIntStatus                             
0     00013057  USBEndpointDataPut                       
0     000130ab  MemCfg_getInitStatus                     
0     000130fe  USBRingBufWrite                          
0     00013151  MemCfg_setLSRAMMasterSel                 
0     000131a3  ConfigDescAlloc                          
0     000131f4  f_opendir                                
0     00013245  SFRA_GUI_lifePulseTsk                    
0     00013294  USBHSCSIInquiry                          
0     000132e3  USBHostEndpointStatusClear               
0     00013380  USBDBulkPacketWrite                      
0     0001341c  USBHSCSIReadCapacity                     
0     00013469  USBHSCSIRequestSense                     
0     000134b5  USBHSCSITestUnitReady                    
0     0001354b  USBDevEndpointDataAck                    
0     000135de  Interrupt_disable                        
0     0001366e  configureCMPSS                           
0     000136b6  configurePWM_1chUpCnt                    
0     00013746  USBEndpointDataAvail                     
0     0001378d  SysCtl_getClock                          
0     000137d3  USBDCDConfigDescGet                      
0     00013817  MemCfg_initSections                      
0     0001385a  USBBufferEventCallback                   
0     0001389d  USBHostEndpointDataAck                   
0     000138e0  USBRingBufAdvanceWrite                   
0     00013923  USBHostAddrSet                           
0     00013965  Interrupt_initModule                     
0     000139a6  USBEndpointDataToggleClear               
0     000139e6  USBHostRequestINClear                    
0     00013a66  GPIO_setPadConfig                        
0     00013aa5  USBEndpointStatus                        
0     00013ae4  USBHostRequestIN                         
0     00013c10  USBIntEnableControl                      
0     00013c4b  USB0DualModeIntHandler                   
0     00013cbe  USBIntStatusControl                      
0     00013d2e  SFRA_GUI_getCmdByte                      
0     00013d65  USBHostPwrConfig                         
0     00013dd0  RxHandler                                
0     00013e6e  Interrupt_enable                         
0     00013ea2  USBBufferInit                            
0     00013ed6  USBHCDPowerConfigSet                     
0     00013f3e  USBHSCSIRead10                           
0     00013f71  SysCtl_selectOscSource                   
0     00013fa3  USBHSCSIWrite10                          
0     00013fd5  ConfigDescFree                           
0     00014031  USBDCDConfigGetInterfaceEndpoint         
0     00014062  USBDeviceEnumResetHandler                
0     00014093  __TI_decompress_lzss                     
0     000140c4  f28x_USB0DeviceIntHandler                
0     000140f5  f28x_USB0DualModeIntHandler              
0     00014126  f28x_USB0HostIntHandler                  
0     00014157  f28x_USB0OTGModeIntHandler               
0     00014188  GPIO_setPinConfig                        
0     000141b8  InternalUSBRegisterTickHandler           
0     000141e8  USBHCDReset                              
0     00014273  USBHCDSetAddress                         
0     000142a0  USBHCDSetConfig                          
0     000142cd  DLOG_4CH_F_init                          
0     000143a9  USBDCDDeviceInfoInit                     
0     000143d5  USBDeviceResumeTickHandler               
0     00014401  USBRingBufInit                           
0     00014458  InternalUSBStartOfFrameTick              
0     00014483  SFRA_GUI_getData                         
0     000144ae  USBDescGet                               
0     000144d9  USBHMSCBlockRead                         
0     00014504  USBHMSCBlockWrite                        
0     0001452f  __TI_auto_init_nobinit_nopinit           
0     00014584  SFRA_GUI_echoCmdByte                     
0     000145ae  SFRA_GUI_echoSizeByte                    
0     000145d8  __c28xabi_cmpd                           
0     00014602  SFRA_GUI_setData32                       
0     0001462b  USBBD_initUSB                            
0     000146a6  C$$EXIT                                  
0     000146a6  abort                                    
0     000146a8  exit                                     
0     000146cf  Device_enableUnbondedGPIOPullups         
0     000146f7  USBBufferInfoGet                         
0     0001471f  USBDBulkRxPacketAvailable                
0     00014747  Device_enableUnbondedGPIOPullupsFor100Pin
0     0001476e  USBDescGetNum                            
0     00014794  __SFRA_F32_inject                        
0     000147df  InternalUSBTickInit                      
0     00014804  SFRA_GUI_echoDataByte                    
0     00014829  USBDCDConfigDescGetNum                   
0     0001484e  USBGPIOEnable                            
0     00014873  XBAR_setEPWMMuxConfig                    
0     00014898  XBAR_setOutputMuxConfig                  
0     000148e1  USBRingBufContigFree                     
0     00014905  disk_write                               
0     00014929  FCL_initADC                              
0     0001494c  __c28xabi_dtof                           
0     0001496f  GPIO_setMasterCore                       
0     00014991  GPIO_setQualificationMode                
0     000149f8  Interrupt_initVectorTable                
0     00014a19  SCI_setConfig                            
0     00014a3a  USBHostReset                             
0     00014a5b  USBHostResume                            
0     00014a7c  USBOTGSessionRequest                     
0     00014a9d  USBStackModeSet                          
0     00014abe  GPIO_setDirectionMode                    
0     00014ade  SFRA_GUI_cmdInterpreter                  
0     00014b1e  USBRingBufAdvanceRead                    
0     00014b5d  InternalUSBHCDSendEvent                  
0     00014b7c  SPI_setConfig                            
0     00014b9b  USBHCDHubDeviceDisconnected              
0     00014bd9  Device_initGPIO                          
0     00014bf7  SCIwrite                                 
0     00014c15  SPI_clearInterruptStatus                 
0     00014c33  Device_init                              
0     00014c50  SFRA_GUI_getDataByte                     
0     00014c6d  SFRA_GUI_getSizeByte                     
0     00014c8a  CLA_setTriggerSource                     
0     00014cc2  SCI_clearInterruptStatus                 
0     00014cde  SFRA_GUI_packWord                        
0     00014cfa  USBIntEnableEndpoint                     
0     00014d16  ramper                                   
0     00014d32  __c28xabi_ftod                           
0     00014d4e  memcpy                                   
0     00014d6a  configureCMPSSFilter                     
0     00014d85  A0                                       
0     00014d9f  SCI_enableInterrupt                      
0     00014db9  USBBufferDataWritten                     
0     00014dd3  USBDCDStallEP0                           
0     00014ded  USBDescGetInterface                      
0     00014e07  USBEndpointDMADisable                    
0     00014e21  USBRingBufUsed                           
0     00014e55  USBDBulkTxPacketAvailable                
0     00014e6e  USBDCDConfigDescGetSize                  
0     00014e87  USBDCDConfigGetInterface                 
0     00014ea0  USBRingBufContigUsed                     
0     00014f01  SPI_enableInterrupt                      
0     00014f19  USBIntStatusEndpoint                     
0     00014f31  B0                                       
0     00014f48  C0                                       
0     00014f5f  FCL_initPWM                              
0     00014fa4  USBDevDisconnect                         
0     00014fbb  USBDevMode                               
0     00014fd2  USBHCDEvents                             
0     00014fe9  USBHostMode                              
0     00015000  USBHostPwrDisable                        
0     00015017  USBHostPwrEnable                         
0     0001502e  USBHostRequestStatus                     
0     00015045  USBModeGet                               
0     0001505c  USBOTGMode                               
0     00015073  disk_read                                
0     0001508a  _c_int00                                 
0     000150a1  CMPSS_configFilterHigh                   
0     000150b7  CMPSS_configFilterLow                    
0     000150cd  USBDevConnect                            
0     000150e3  USBRingBufFlush                          
0     000150f9  f_mount                                  
0     0001510f  setupCpuTimer                            
0     0001513a  SysCtl_getLowSpeedClock                  
0     0001514f  USBRingBufFree                           
0     00015179  USBHCDRegisterDrivers                    
0     0001518d  USBHostSuspend                           
0     000151a1  strncpy                                  
0     000151b5  Cmd_pwd                                  
0     000151c8  GPIO_setAnalogMode                       
0     000151db  USBBufferFlush                           
0     000151ee  USBBufferSpaceAvailable                  
0     00015201  USBDevAddrSet                            
0     00015214  memcmp                                   
0     00015239  USB0DeviceIntHandler                     
0     0001524b  USB0HostIntHandler                       
0     0001525d  USBDescGetInterfaceEndpoint              
0     00015281  SFRA_GUI_setButton                       
0     00015292  SFRA_GUI_setSlider                       
0     000152a3  SFRA_GUI_setText                         
0     000152b4  USBHCDPowerConfigInit                    
0     000152c5  USBHHubEnumerationComplete               
0     000152d6  USBHHubEnumerationError                  
0     000152e7  USBHMSCDriveOpen                         
0     000152f8  USBNumEndpointsGet                       
0     00015309  B1                                       
0     00015319  MSCCallback                              
0     00015329  OTGDeviceDisconnect                      
0     00015379  SFRA_GUI_runSerialHostComms              
0     00015388  __c28xabi_subd                           
0     00015396  C1                                       
0     000153bd  USBHHubInit                              
0     000153ca  TxHandler                                
0     000153d6  _args_main                               
0     000153e2  USBHCDPowerAutomatic                     
0     000153ed  strcmp                                   
0     000153f7  __TI_decompress_none                     
0     000153ff  strcat                                   
0     00015407  tformat_checkCRC                         
0     0001540f  SCIprintf                                
0     0001542b  A2                                       
0     00015431  A3                                       
0     00015437  B2                                       
0     0001543d  B3                                       
0     00015443  C2                                       
0     00015449  C3                                       
0     0001544f  CPUTimer_setEmulationMode                
0     00015455  __TI_zero_init                           
0     0001545b  memset                                   
0     00015466  SFRA_GUI_spareTsk08                      
0     00015493  FCL_initQEP                              
0     0001549b  ModeCallback                             
0     0001549f  __error__                                
0     000154a2  FCL_getSwVersion                         
0     000154a8  _system_pre_init                         
0     000154aa  FCL_runPICtrl                            
0     000155c8  FCL_runPICtrlWrap                        
0     0001568d  FCL_resetController                      
0     000156c6  SysCtl_delay                             
0     00019000  g_eState                                 
0     00019001  g_eUIState                               
0     0001944a  g_pui8USBRxBuffer                        
0     0001954a  g_pui8USBTxBuffer                        
0     0001964a  tformatCRCtable                          
0     0001974a  g_psDCDInst                              
0     00019780  speedWePrev                              
0     00019782  curA_PPBRESULT                           
0     00019784  curB_PPBRESULT                           
0     00019786  curC_PPBRESULT                           
0     00019788  voltDC_PPBRESULT                         
0     0001978a  AdcIntFlag                               
0     0001978c  pwmCompA                                 
0     0001978e  pwmCompB                                 
0     00019790  pwmCompC                                 
0     00019792  clarke1                                  
0     0001979c  park1                                    
0     000197aa  D_cpu                                    
0     000197c0  svgen1                                   
0     000197d2  pi_id                                    
0     00019800  FCL_params                               
0     000198aa  g_pHCDPool                               
0     0001992a  clMagVect                                
0     0001998e  clPhaseVect                              
0     000199f2  freqVect                                 
0     00019a56  olMagVect                                
0     00019aba  olPhaseVect                              
0     00019b1e  plantMagVect                             
0     00019b82  plantPhaseVect                           
0     00019bf8  SFRA_GUI_cmdPacket                       
0     00019bfe  g_ppsDevInfo                             
0     00019c00  tFormat_dataId                           
0     00019c02  Alpha_State_Ptr                          
0     00019c04  A_Task_Ptr                               
0     00019c06  B_Task_Ptr                               
0     00019c08  C_Task_Ptr                               
0     00019c0a  offset_SDFM1                             
0     00019c0c  offset_SDFM2                             
0     00019c0e  tformatAngle                             
0     00019c10  tformatSpd                               
0     00019c12  retVal1                                  
0     00019c14  crcResult                                
0     00019c16  position                                 
0     00019c18  turns                                    
0     00019c1a  speed1                                   
0     00019c40  dlog_4ch1                                
0     00019c5a  SFRA_GUI_commsOKflg                      
0     00019c5b  SFRA_GUI_serialCommsTimer                
0     00019c5c  SFRA_GUI_lowByteFlag                     
0     00019c5d  SFRA_GUI_sendTaskPtr                     
0     00019c5e  SFRA_GUI_rxChar                          
0     00019c5f  SFRA_GUI_rxWord                          
0     00019c60  SFRA_GUI_taskDoneFlag                    
0     00019c61  SFRA_GUI_numWords                        
0     00019c62  SFRA_GUI_wordsLeftToGet                  
0     00019c63  SFRA_GUI_dataOut16                       
0     00019c64  SFRA_GUI_rcvTskPtrShdw                   
0     00019c65  SFRA_GUI_delayer                         
0     00019c66  SFRA_GUI_memGetPtr                       
0     00019c67  SFRA_GUI_memGetAmount                    
0     00019c68  SFRA_GUI_memSetPtr                       
0     00019c69  SFRA_GUI_led_flag                        
0     00019c6a  SFRA_GUI_led_gpio                        
0     00019c6b  SFRA_GUI_sweep_start                     
0     00019c6c  SFRA_GUI_rcvTaskPointer                  
0     00019c6e  SFRA_GUI_sci_base_addr                   
0     00019c70  SFRA_GUI_dataOut32                       
0     00019c72  SFRA_GUI_memDataPtr16                    
0     00019c74  SFRA_GUI_memDataPtr32                    
0     00019c76  SFRA_GUI_memGetAddress                   
0     00019c78  SFRA_GUI_memSetValue                     
0     00019c7a  SFRA_GUI_temp                            
0     00019c80  tformatData                              
0     00019da6  g_pfnTickHandlers                        
0     00019dfe  SFRA_GUI_arrayGetList                    
0     00019e1e  SFRA_GUI_cmdDispatcher                   
0     00019e3e  SFRA_GUI_dataSetList                     
0     00019e5e  SFRA_GUI_varGetList                      
0     00019e7e  SFRA_GUI_varSetBtnList                   
0     00019e9e  SFRA_GUI_varSetSldrList                  
0     00019ebe  SFRA_GUI_varSetTxtList                   
0     00019ede  sfra1                                    
0     00019f0a  g_pvTickInstance                         
0     00019f16  g_eOTGModeState                          
0     00019f18  g_ui32PollRate                           
0     00019f1c  g_eCurrentUSBMode                        
0     00019f1e  g_pcStatus                               
0     0001a362  DBUFF_4CH1                               
0     0001a4f2  DBUFF_4CH2                               
0     0001a682  DBUFF_4CH3                               
0     0001a812  DBUFF_4CH4                               
0     0001a9a2  g_pui8BulkDeviceDescriptor               
0     0001a9b4  g_pui8BulkDescriptor                     
0     0001a9be  _lock                                    
0     0001a9c0  serialCommsTimer                         
0     0001a9c1  offsetCalCounter                         
0     0001a9c2  hlt                                      
0     0001a9c3  llt                                      
0     0001a9c4  clkPrescale                              
0     0001a9c5  sampWin                                  
0     0001a9c6  thresh                                   
0     0001a9c7  LEM_curHi                                
0     0001a9c8  LEM_curLo                                
0     0001a9c9  SHUNT_curHi                              
0     0001a9ca  SHUNT_curLo                              
0     0001a9cb  enableFlag                               
0     0001a9cc  backTicker                               
0     0001a9cd  tripFlagDMC                              
0     0001a9ce  clearTripFlagDMC                         
0     0001a9cf  runMotor                                 
0     0001a9d0  ledCnt1                                  
0     0001a9d1  speedLoopPrescaler                       
0     0001a9d2  speedLoopCount                           
0     0001a9d3  lsw2EntryFlag                            
0     0001a9d4  FCL_cycleCount                           
0     0001a9d5  fclClrCntr                               
0     0001a9d6  fclCycleCountMax                         
0     0001a9d7  posPtrMax                                
0     0001a9d8  posPtr                                   
0     0001a9d9  sfraTestLoop                             
0     0001a9da  tFormat_encCmdStatus                     
0     0001a9db  tFormat_crcError                         
0     0001a9dc  offset_lemV                              
0     0001a9de  offset_lemW                              
0     0001a9e0  offset_lemU                              
0     0001a9e2  offset_IP                                
0     0001a9e4  offset_DcImcu                            
0     0001a9e6  K1                                       
0     0001a9e8  K2                                       
0     0001a9ea  curLimit                                 
0     0001a9ec  isrTicker                                
0     0001a9ee  fclLatencyInMicroSec                     
0     0001a9f0  maxModIndex                              
0     0001a9f2  T                                        
0     0001a9f4  VdTesting                                
0     0001a9f6  VqTesting                                
0     0001a9f8  IdRef                                    
0     0001a9fa  tempIdRef                                
0     0001a9fc  IqRef                                    
0     0001a9fe  speedRef                                 
0     0001aa00  lsw1Speed                                
0     0001aa02  alignCntr                                
0     0001aa04  alignCnt                                 
0     0001aa06  alignInitCnt                             
0     0001aa08  IdRef_start                              
0     0001aa0a  IdRef_run                                
0     0001aa0c  posCntr                                  
0     0001aa0e  posCntrMax                               
0     0001aa10  posSlewRate                              
0     0001aa12  dlogCh1                                  
0     0001aa14  dlogCh2                                  
0     0001aa16  dlogCh3                                  
0     0001aa18  dlogCh4                                  
0     0001aa1a  sfraCollectStart                         
0     0001aa1c  sfraNoiseD                               
0     0001aa1e  sfraNoiseQ                               
0     0001aa20  sfraNoiseW                               
0     0001aa22  angMax                                   
0     0001aa24  ipark1                                   
0     0001aa40  rc1                                      
0     0001aa50  tFormat                                  
0     0001aa60  pi_pos                                   
0     0001aa80  spdObs                                   
0     0001aa9a  pid_pos                                  
0     0001aac0  pid_spd                                  
0     0001aae8  posEncElecTheta                          
0     0001aaf6  adcHandle                                
0     0001ab00  cm1_const                                
0     0001ab10  cm1                                      
0     0001ab24  volt1                                    
0     0001ab40  se1_const                                
0     0001ab58  se1                                      
0     0001ab80  fe1_const                                
0     0001abc0  fe1                                      
0     0001ac06  g_sFresultStrings                        
0     0001ac3e  g_psMSCInstance                          
0     0001ac40  g_sTxBuffer                              
0     0001ac5c  g_sRxBuffer                              
0     0001ac80  g_sBulkDevice                            
0     0001acf4  g_psCmdTable                             
0     0001ad2a  tformat_tile1HLCInstr                    
0     0001ad4a  posEncMechTheta                          
0     0001ad68  g_ui32TxCount                            
0     0001ad6a  g_ui32RxCount                            
0     0001ad6c  g_ui32Flags                              
0     0001ad6e  Example_Result                           
0     0001ad70  Example_PassCount                        
0     0001ad72  Example_Fail                             
0     0001ad74  pwmHandle                                
0     0001ad7a  __TI_enable_exit_profile_output          
0     0001ad7c  __TI_cleanup_ptr                         
0     0001ad7e  __TI_dtors_ptr                           
0     0001ad80  g_bUSBTimerInitialized                   
0     0001ad82  g_ui32CurrentUSBTick                     
0     0001ad84  g_ui32USBSOFCount                        
0     0001ad86  g_psBulkSections                         
0     0001ad8a  g_iUSBMode                               
0     0001ad8c  g_ui32WaitTicks                          
0     0001ad8e  vTimer0                                  
0     0001ad92  vTimer1                                  
0     0001ad96  vTimer2                                  
0     0001ad9c  errno                                    
0     0001b844  g_pui8ConfigString                       
0     0001b874  g_pui8DataInterfaceString                
0     0001b89c  g_pui8ProductString                      
0     0001b8c4  g_pui8ManufacturerString                 
0     0001b8e8  g_pui8BulkInterface                      
0     0001b900  g_sBulkConfigSection                     
0     0001b904  g_sBulkInterfaceSection                  
0     0001b908  g_sBulkConfigHeader                      
0     0001b90c  g_sBulkHandlers                          
0     0001b93e  g_pui8SerialNumberString                 
0     0001b95c  g_ppui8StringDescriptors                 
0     0001b974  g_sUSBEventDriver                        
0     0001b980  g_sUSBHostMSCClassDriver                 
0     0001b988  g_pui8LangDescriptor                     
0     0001b98c  g_ppBulkConfigDescriptors                
abs   00000100  CLA_SCRATCHPAD_SIZE                      
abs   00000380  __TI_STACK_SIZE                          
abs   ffffffff  __TI_pprof_out_hndl                      
abs   ffffffff  __TI_prof_data_size                      
abs   ffffffff  __TI_prof_data_start                     
n/a   UNDEFED   __c_args__                               

[571 symbols]
